:020000040001F9
:10600000D03F0020756101008F6101005D620100D9
:106010000000000000000000000000000000000080
:10602000000000000000000000000000936101007B
:106030000000000000000000956101009761010070
:10604000996101009961010099610100C1F50100A8
:1060500099610100000000009DFA0100659E0100A9
:106060009961010099610100CDBF010099610100B2
:106070009961010099610100996101009961010034
:10608000996101001BDD0100996101009961010026
:1060900031DD01009961010057E5010099610100BE
:1060A00099610100996101000000000000000000FA
:1060B00000000000000000000000000000000000E0
:1060C000034885460AF086FE00480047476D0100F8
:1060D000D03F0020401E00BF00BF00BF00BF00BF78
:1060E00000BF00BF00BF00BF00BF00BF00BFF1D1B5
:1060F00070470000401E00BF00BF00BF00BF00BFD0
:1061000000BF00BF00BF00BF00BF00BF00BFF1D194
:1061100070470000401E00BF00BF00BF00BF00BFAF
:1061200000BF00BF00BF00BF00BF00BF00BFF1D174
:1061300070470000401E00BF00BF00BF00BF00BF8F
:1061400000BF00BF00BF00BF00BF00BF00BFF1D154
:1061500070470000401E00BF00BF00BF00BF00BF6F
:1061600000BF00BF00BF00BF00BF00BF00BFF1D134
:10617000704700000321094802680A43026008488A
:1061800002680A4302600748804707480047FEE765
:10619000FEE7FEE7FEE7FEE7FEE70000240500401D
:1061A00054050040B5610100C16001002349224847
:1061B0000860704710B500F01DF8002805D021498F
:1061C0001F484860C813204988612048018CC9B223
:1061D00001290ED1818C09070BD1018D0906090F08
:1061E000042906D1808D0006000F02D11849012034
:1061F000886010BD1548018CC9B2012917D1818C66
:10620000090714D1018D09060A0F03D1828D1206E8
:10621000120F0ED0090F012903D1828D1206120F21
:1062200007D0032903D1808D0006000F01D0002084
:1062300070470120704700000024F4000020002077
:10624000DFFF07C000050040006C0040C00F00F0F9
:106250000006004004F048F900F035FE04F044F96F
:1062600000F031FE04F040F900F02DFE04F03CF99E
:1062700000F029FE7CB5FE4C08280CD00A2838D145
:10628000606B07F07FFEA08AFA49884225D1002280
:106290000521090424E0684601F0D3FC6846007833
:1062A000002807D03C210D1A7D20C0004543012065
:1062B000207100E0F04D206B07F064FEFF23690CB5
:1062C000E803F5330022C01851415A0000230AF0B8
:1062D000F7FC01460022206B03E000220121C903E4
:1062E000606B07F0E5FD002803D004F0FDF800F036
:1062F000EAFD7CBD10B574DF002803D004F0F4F88B
:1063000000F0E1FD10BD10B5D94C0120A07204F0E1
:10631000EBF801F0E6FEA08AD649884202D01321AC
:1063200076DF06E0206A002803D0FFF7E3FF0020B5
:106330002062CF48133008F01CFD606B07F022FE8E
:10634000206B07F01FFE02F037F800200AF03CFC3B
:1063500000200AF025FC01F021FE10BD7CB503F001
:10636000C6FD0025C24C002810D1607A00280DD04F
:10637000A07B401CC0B2A073022809D3E07A002899
:1063800006D10120E072FFF7BEFF7CBDA573E57268
:1063900001F054FC0122694601F0A7FC012001F044
:1063A00051FD0646400709D501F05AFC03F07EFE78
:1063B00004F06EFA0021012004F0EEFFF00705D092
:1063C00004F0E1F90021022004F0E6FFB00701D556
:1063D00003F007FFA64844300079002804D0607A13
:1063E000002801D0012000E000200AF0D9FB03F0D2
:1063F00056FD684603F064FE20790028C5D0206B66
:1064000007F0C0FD0F2100224904206B07F050FD6A
:10641000002803D004F068F800F055FD25717CBD1C
:1064200010B50068002806D001280BD0022801D141
:1064300003F0D0FE10BD0020FFF790FF0820FFF70B
:1064400019FF10BD03F032FE10BD7047F8B50446C9
:106450004279214689480831854D012A15D0032A01
:1064600012D106463278401C10187C220270401C63
:10647000E2880AF055FC3078A17940183070E8695C
:10648000012109040843E861F8BD7C4BAE7C01277B
:106490005B1C7B4A012E0DD0042EF5D1977302258B
:1064A000176055609360A2790270401CE2880AF080
:1064B00037FCF8BD9773176057609360A27902703C
:1064C000401CE2880AF02CFCD9E708B501680029D5
:1064D00008D0012907D003291CD0042902D1083093
:1064E000FFF7B4FF08BD624869462C3008F0A3FBF3
:1064F00000280BD10098002802D000F0F3FC08BD62
:106500005B482C3008F06FFB0028F8D003F0ECFF5C
:1065100000F0D9FC5649807A887408BD544900209F
:1065200088722DDF704770B5514C0546206C07F01E
:1065300029FD002D0BD000225249206C07F0B8FC39
:1065400001F0E7FF002009F0BBFE0C2000E00D2069
:1065500000F020FF70BD01B501226946402004F023
:10656000E3FE08BD71B5ABB0002420A90C7740480C
:1065700028A9427C097B8A4250D0417428A871DF47
:10658000002847D110A81E94848718A804760124F7
:10659000447600201EAD28A90622131A2E18401C8E
:1065A000CB5CC0B2B3700628F7D33C2168460AF032
:1065B000D0FB02200090684604812BA8269503900A
:1065C000082120A8818224A80C903C210FA80AF061
:1065D000C0FB27A8DF211390C94320A80180847045
:1065E0002949818029498471487B0A7B0102114332
:1065F00020A8018121481038017B20A88172032145
:1066000010A8018320A817900FA9684607F07EF80C
:10661000002803D003F068FF00F055FC2CB070BDDB
:1066200030B5134C87B0606B07F0ACFCA07A002843
:1066300009D105A806F029FF002843D105980028B4
:1066400003D00120E07007B030BD142168460AF085
:1066500080FB0748002544304079002821D0A08ADB
:10666000044988421DD00420FFF77CFF03210FE07E
:1066700004200020FFFF000060EA0000FC2B002047
:10668000C42E00208F020000E7FE000082230200DB
:106690006846017001950572FB490182458273DFEE
:1066A0000EE00520FFF75EFF684605700195057254
:1066B000332101821421418202202062684673DF67
:1066C0000028C0D003F010FF00F0FDFBA8E73EB5A6
:1066D000EE4C207B032831D1002569460D700195D1
:1066E0006846029501F079FE04E001A801F094FEED
:1066F0006D1CEDB2684600788542F6D3E17BE34835
:106700004B30002911D0217C4171207C401C207429
:10671000DE48062201A957300AF002FBDB491222AB
:106720004B31DB4806F033F904E0062201A9801D55
:106730000AF0F6FAE07B01214840E0733EBDD34801
:10674000C169FF2201321143C1617047CF4881798D
:10675000491C8171C169012252021143C161704714
:1067600010B58AB0684671DF00284CD16A4690782F
:10677000517800020843C7490AF078FA0846C3492D
:106780000024C882039404940594C3A2069406CA04
:10679000039104920A210AF069FA30316A461176AF
:1067A0000A210AF063FA30316A46D1750A210AF0EB
:1067B0005DFA30316A469175303050752D20107574
:1067C0001120107203A80AF0CFFA82B203A902A81E
:1067D0007CDF002817D15120800178DF002812D1FA
:1067E0000794282168460894818319214901C183AF
:1067F000FF210484F531418407A87ADF002802D103
:1068000077DF002803D003F06FFE00F05CFB0AB0D6
:1068100010BD10B50068002809D19C483B21808A32
:1068200076DF002803D003F05FFE00F04CFB10BDC4
:1068300003F05AFE00F047FB70B50C460A460546C9
:1068400001469348383005F07FFE2178112905D1A3
:106850008E48042229462C300AF062FA002070BDCE
:1068600070B58A4A0188443200255279874C19292B
:106870003FD00ADC102918D011291DD0152903D0CA
:10688000172901D100F02EFB70BD80483929808A7C
:1068900003D0522929D05529F6D1132176DF0028BB
:1068A000F2D003F021FE00F00EFB8088A08229E0E8
:1068B0000A20FFF7DFFC70BD207B032802D10020F7
:1068C000FFF731FE207B012802D10B2000F062FD92
:1068D00000202573C043A082256274DFE0690007B1
:1068E000800FE8D1FFF79CFE70BD00221146A9DFA2
:1068F000D5E780790028F7D16448256218304078C0
:106900000028D5D1002AD3D170BD08B5684606F05D
:10691000BCFD002803D003F0E7FD00F0D4FA009896
:10692000002803D059490120487008BD2DDF08BD5B
:1069300008B5684606F0A9FD002803D003F0D4FD91
:1069400000F0C1FA0098002803D050490120887057
:1069500008BDB1203CDF2DDF08BD10B5044608F0AE
:10696000FDFB21464A4805F0B3FF4948214638302F
:1069700005F0F2FD46482146203006F0ABF82046EF
:1069800007F0FAFC2046FFF76BFF10BD10B5044678
:1069900006F00BFB204600F0C8FB10BDF0B500254B
:1069A00085B00446049500952E460295032801D033
:1069B000042C3FD13B4F012923D0684607F029FB27
:1069C000324802AA4079C000C0194168009807F017
:1069D00025FB032C2D4C344861792FD0012967D039
:1069E000029981420CD8E06B07F0CCFAE5712F4890
:1069F0000299814277D8FF260136A06B07F0C2FAD0
:106A000076E0224EF079002806D101210022C90348
:106A1000F06B07F04DFA3472F079401CF071B571EB
:106A200004A807F0F6FA0498032C05D0B860B06B00
:106A300007F0A8FA05B0F0BD3860F8E7002938D0B3
:106A40000299814212D8E06B07F09CFAE571174871
:106A50000299814205D8FF260136A06B07F092FA11
:106A600004E0A06B07F08EFA0126B602E079012857
:106A700034D102AA3968009807F0D0FA01200299AF
:106A8000C00381421FD223E016080000042000202A
:106A9000B42B00201027000042726163656C6935D9
:106AA0000000000084230020291C00008F02000049
:106AB0002CE002AA3968009807F0B0FA0120029988
:106AC000C003814201D3E57108E0E079012805D1D6
:106AD000E06B07F057FAFF26E57101360098786001
:106AE00065712CE0FFE7A06B07F04CFA0126F60277
:106AF000E07901281FD102AAB968009807F08EFA40
:106B000001200299C00381420AD20EE002AAB968AC
:106B1000009807F083FA01200299C003814201D353
:106B2000E57108E0E079012805D1E06B07F02AFA69
:106B3000FF26E57101360098F86001206071002E93
:106B400000D177E7FE48C1693143C16172E703298B
:106B500006D1072804D1FA48C16940221143C16116
:106B6000704770B5001F00250122F54C03000AF0A4
:106B700083F908050709090E14170E06626270BD35
:106B8000656270BDC8B2A26203F069FD70BD0420E9
:106B9000A062C8B203F063FDF2E701F0DAFC70BD59
:106BA00001F0B7FC70BD70471CB50446684601F0A3
:106BB00048F868467D21C088C9000AF057F821705E
:106BC0006846007960706846C078A0706846807832
:106BD000E0706846407820711CBDD94910B5443139
:106BE000497800290BD001280AD0D648007800281F
:106BF00003D0D5480068042801D101F072FA10BD15
:106C0000CF48416A0029FAD1C0690028F7D1042091
:106C100000F0C0FB10BD38B5C94CE0694006E06922
:106C200005D540218843E06100F066F938BDC00316
:106C3000E06909D5012109048843E061606A002800
:106C4000F4D100F0CBFC38BD8006E06907D52021E7
:106C50008843E061BA48133008F08BF838BD8107EB
:106C6000B748E169808A05D502229143E161132189
:106C700076DF38BD4A07B5490CD58842F9D1E069BD
:106C800004218843E06103F02FFC01F02AFAFFF7AA
:106C90003CFE38BDE269120710D58842F9D1E0699F
:106CA00008218843E0612021A9480AF052F803F046
:106CB0001BFC01F016FAFFF73BFE38BDE069C0058A
:106CC0000AD50321162000F006F9E069FF21013101
:106CD0008843E06102201AE0E0698005E06919D587
:106CE000012149028843E061E07A617A0842E4D1F7
:106CF000012002460090002332213C2001F065FA79
:106D0000A07A002802D0FFF709FC38BD032000F06C
:106D100041FB38BD4005E06905D501218902884362
:106D2000E0610020F3E7000506D5E0690121C90212
:106D30008843E0610120EAE70020E06106F08EFE72
:106D400000F05EFA38BD834888B00125456000F048
:106D500025F900F064F98049022008F0F9FE0028C6
:106D60007DD100F03FFF002879D000F0FAFC03F05D
:106D7000CBFE04F0E3FF01F080F900286FD001F0B2
:106D800015FA00286BD001F0F1FA00287ED000F04F
:106D9000F0FA00287AD003F0C9FA002876D06F49BB
:106DA000032008606E4E6C07B460FF202D3008F0A1
:106DB00045FEF46000F0DDF96A4A1421082006F06F
:106DC000C3FD002862D100F080F9FFF7C9FC00F094
:106DD00053F90520FFF7C6FB1C21684609F0B9FFEF
:106DE000711301910F21090400200291009069465E
:106DF0000D73594928318A896946CA8108745A48ED
:106E000005905A480690684607F061FA00283DD17F
:106E100003F07AFE01F0B1FA494C002803D1607BFF
:106E200002210843607303F010F9002802D1607B4F
:106E30002843607304F0C3FD002803D1607B042164
:106E40000843607308F050FF494809F06EFE494856
:106E500009F078FE484809F06FFE484800E015E068
:106E600009F0E3FE03F022F903F0B4F900F0CAFEE2
:106E700000280BD0FFF7D4FB03F011F830480022B4
:106E80000121603000F010FE002803D003F02CFB3D
:106E900000F019F800F034FE00F08DF9E0694021AF
:106EA0000843E0610820FFF7E5F9082000F072FAD6
:106EB000E069002802D0FFF7AEFEF9E706F0CEFD4C
:106EC00000F09EF9F4E7BFF34F8F2E492C48C860BD
:106ED000BFF34F8FFEE7214A89008000743A801883
:106EE000016070471C4810B5603005F02EFC1A4850
:106EF000603005F034FC10BD08B519480069000683
:106F0000C00F00D001200E494A7A904206D0487244
:106F1000002804D002F0C3FF04F05CFF08BD887AAB
:106F2000002801D0FFF7FAFA002009F04DFE0020FA
:106F300009F036FE0320002301221921490123E034
:106F40000420002090200020A0200020FFFF00004F
:106F5000D42E0020400500408C2B002074070050E8
:106F6000000500503C2A0020136801003168010030
:106F7000636B0100A76B0100A96B0100DB6B0100D3
:106F80000400FA0500ED00E00090FF202D3001F034
:106F90001CF900211E2004F0E1FE08BDF8B5002414
:106FA000C84FC94E0325142C2CD00EDC112C1DD03B
:106FB00006DC052C1CD0062C1AD0072C16D119E0A3
:106FC000122C13D0132C11D122E0204616380300C6
:106FD00009F052FF09100C0C0C0E0E0C0C060C00E4
:106FE000B848783005600120800716E0012102E0F2
:106FF000002100E003212046FFF76DFF641C202CD8
:10700000D1D3F8BD01212046FFF765FF641CCAE714
:10701000A000C01905600120A040B060EEE708B5EF
:10702000AA480090AA4B0E220D21002006F0A6FED1
:10703000002803D003F058FAFFF745FFA54A0121C5
:10704000A54806F0EEFEA448A44A0021001D06F063
:10705000E8FEA148A24A0121103006F0E2FE9E4857
:10706000A04A0021083006F0DCFE9B489E4A002121
:107070000C3006F0D6FE08BD00B59C4887B04268CB
:10708000016801920091C26881680392029141698E
:1070900000690591049004A9954805F0C2FA0028FA
:1070A0000DD193486946383805F048FC002806D1D0
:1070B0008F4802A9183805F080FD002803D003F09E
:1070C00013FAFFF700FF07B000BD1FB505F0D4FFAE
:1070D000002825D16946087303A807F0F3FC0028AF
:1070E0001ED101A80621023009F033FE1E20694698
:1070F000C880087A01221043E12108400C30DF21CA
:107100000840694608720720487210208872794842
:10711000009071480A711D3807F02BFD002803D03C
:1071200003F0E2F9FFF7CFFE1FBD10B5022801D032
:10713000032808D16848002130380278002A03D09B
:10714000017000F081F810BD4278002A03D0417030
:10715000FFF7DBFB10BD8278002A03D08170FFF7B8
:10716000E7FB10BDC278002AFBD0C170FFF758FAC8
:1071700010BD08B560490120C863002350225F4953
:10718000082007F0BBF9002810D16946009008706C
:10719000684660DF002809D1594807F0CCF900287B
:1071A00004D1584807F0CFF9002803D003F09CF928
:1071B000FFF789FE08BD484810B5534BC522022190
:1071C0003C3007F05CFA002803D107F087FA00286A
:1071D00003D003F089F9FFF776FE03220021104661
:1071E00000F017F803220021042000F012F83848BC
:1071F000103806F00EFF3648083806F00AFF10BDBA
:1072000010B540DF002803D003F06EF9FFF75BFEF6
:1072100010BD120489000A432A4980004018026008
:1072200070471CB501910090384A0821684606F065
:107230009FFB1CBD1CB50090684601714271344A29
:10724000082106F095FB1CBD08B5684606F01DF93F
:10725000002819D10098002804D01F490120303996
:10726000087008BD022200210520FFF7D2FF03228B
:1072700000211046FFF7CDFF032200210420FFF775
:10728000C8FF34DF0028ECD003F02EF9FFF71BFE17
:1072900010B50246082903D003F026F9FFF713FEC4
:1072A00011685068884710BD10B50246082903D000
:1072B00003F01AF9FFF707FE517910791268904729
:1072C00010BD0000000700500005005023720100AF
:1072D000942300205D63010034200020CD6601006E
:1072E000CF6601003F6701004D6701008413020073
:1072F000EC2B00203968010040000040EC29002000
:107300005B6901008D690100357201009172010015
:10731000A972010070B5C34800250078C24C00284E
:1073200000D02570A068102800D3A560A068BE49D1
:10733000C000143140182178002911D02178491E4D
:107340002170A2686168914201D0A1686160006803
:10735000804701210022C903E06806F0A9FD70BD45
:1073600000F01CFE00F0BDFEA0680928F7D2A56061
:1073700070BDAD4810B5AD4A00210C3006F051FD8E
:10738000002801D0002010BDA748002181600170B5
:10739000012010BD70B50546A2480078002821D113
:1073A000A14CA068102801D30020A060E06806F07E
:1073B000E9FDA0689C49C00014314618284602F037
:1073C000FFFC002802D171682846884700F086FE3D
:1073D000002801D100F071FE256100229449E06887
:1073E00006F066FD70BDF0B5FFB094B000206946B0
:1073F0001290087208868F4C0D901190A568064671
:10740000002D70D0216800296DD0A0818A480E908F
:10741000FF3001300F90019088480178401C0F1810
:1074200004F0EFF900287DD0B2E00CA9284604F062
:1074300053FA109000280CD0684602AA03A9008EC7
:1074400004F079FA002857D010990020012902D0C1
:1074500006E06D1C9CE06946098E202900D10120C0
:107460006946097B00916946097A002904D10128FF
:107470003AD11198002837D0009840080090802E0B
:1074800010D2301880280DD900998020411A13A8F5
:107490008019119109F05DFC53A88019119909F028
:1074A00058FC8026009830181190FF2801D9A5605B
:1074B00071E00D9903A8411813A88019009A09F0EA
:1074C0002FFC00990D98009A411803A8091853A899
:1074D000801909F025FC119886B2012012906846A7
:1074E000007A119003E076E0129800284ED10098BF
:1074F000102802D020281BD048E0A089FF210830A6
:1075000001318842D3D8A08103A9082201310E9805
:1075100009F006FC05A908220131019809F000FCD8
:107520000E9800E054E008300E90019808302CE0EE
:10753000A089F82801D078280FD10830A08108212F
:107540000E9809F006FC0821019809F002FC0E983B
:1075500008300E90019808300190A089FF2110306A
:1075600001318842A3D8A08103A9102201310E98CD
:1075700009F0D6FB07A910220131019809F0D0FBD0
:107580000E9810300E9001981030019010982D1820
:10759000BD4200D249E71298002815D00020A081F2
:1075A000761E30B2244A53AE0F990BE013AB1B5C2E
:1075B0001370335C0B70A389521C5B1C491C401E6A
:1075C000A38100B20028F1DA04F072F9BD4202D3BF
:1075D0000020A06020607FB014B0F0BD08B5154851
:1075E0004B234068DB00012806D002280AD004F0B3
:1075F000F1FB00F044FE08BD092003226421009045
:10760000C82004E00220024664210090084600F0F1
:10761000DCFD0720FFF7BEFE08BD06480021016023
:10762000816070470E20002090200020157301001B
:10763000CD0C0000C42E0020C42C0020FC2B002008
:10764000F8B50C214843E74E0746801900900179B0
:1076500001242046E44D8840E860F15D20468840E2
:10766000A8602046FEF736FD009801792046884044
:10767000A860E861F05D8440EC61F8BD70B50C2253
:10768000D84E50438219012355681C46D64AAC4057
:107690009461305C8340D36080200E46064201D066
:1076A000946000E0D46000BF00BF00BF00BF9360E3
:1076B00000BF00BF00BF00BFD3604008EDD1D46160
:1076C000936000BF00BF00BF00BF1069D360E840F7
:1076D000C007C017401C946170BDF3B504460C2070
:1076E0004443C048002527183A7901239340BE4AF5
:1076F00081B0D3618026BB480121005D8140BA483A
:10770000816000BF00BF00BF00BF02693B79DA4063
:10771000D20701D03543EDB2C1600120FEF7DAFC9B
:1077200000BF00BF00BF00BF7608E4D13A79012155
:1077300008469040AC4AAB4B9061029E002E01D0AF
:10774000D06000E0906000BF00BF00BF00BF185DC8
:107750008140916000BF00BF00BF00BFD1602846DC
:10776000FEBDF8B59F4E00273772182030601720F5
:1077700070609F499D480862C86101249A4D2006A7
:10778000A861A8604010E8612046FEF7A3FC2869C4
:107790007168C840C00718D120468840A861317878
:1077A00020468840E8600120FEF794FC00BF00BF3F
:1077B00000BF00BF307821468140A9600120FEF75C
:1077C00089FC7F1CFFB2092FE9D33178204688401D
:1077D000A860A861317920468840A860A86100208F
:1077E00030750D20F0600C20814930617F484039B0
:1077F0004863086301204003A861A8604010E86165
:107800000120FEF767FC29693069C140C90719D119
:1078100021468140A9610027317B20468840E860ED
:107820000120FEF757FC00BF00BF00BF00BF307B48
:1078300021468140A9600120FEF74CFC7F1CFFB26D
:10784000092FE9D3317B20468840A860A861317CAC
:1078500020468840A860A861624900202031087055
:107860000820B06109206249F0616048403908622F
:107870004862FF200130A861A8604000E861012053
:10788000FEF728FC2969F069C140C90719D12146D2
:107890008140A9610027317E20468840E8600120B0
:1078A000FEF718FC00BF00BF00BF00BF307E2146BE
:1078B0008140A9600120FEF70DFC7F1CFFB2092F5B
:1078C000E9D3317E20468840A860A861307F84409B
:1078D000AC60AC61F8BDFFB581B01C46150013D09B
:1078E00001980C2148433F49012247183A720198F8
:1078F00000F054F802990198FFF7C0FE060023D06B
:107900000298C0070BD118E0012005B0F0BD002C93
:107910000BD001210198FFF7E0FE28706D1C204676
:10792000641EE4B20028F2D10EE00021F2E72978CB
:107930000198FFF7A3FE06406D1C2046641EE4B2CA
:10794000002801D0002EF2D10A983146814302D19D
:107950000198FFF775FE002038723046D5E7FFB575
:10796000012481B01F4615460E46002907D101208B
:10797000CBE731780198FFF781FE0440761C28465A
:107980006D1EEDB2002801D0002CF2D12046B84384
:1079900002D10198FFF754FE2046B6E7F8B50C2156
:1079A0004843104E07468019009001790124204673
:1079B00088400D4D0146A861F25D20469040A861C7
:1079C000A960A8602046FEF785FB00980179204653
:1079D0008840E8600120FEF77DFBF05D8440EC60AC
:1079E000F8BD0000082F0020000500500C06000024
:1079F0004007005010B54D4A9368002B0BD0047817
:107A00000A46806821469847002803D048A21A21D8
:107A1000FEF720FC10BD022908D001290CD0032953
:107A2000F8D1027883681046984710BD03788268C1
:107A300002211846904710BD027801218368F2E7C1
:107A4000F3B5002481B00F460125384E28E00C2004
:107A50007168604340184178022904D0012909D097
:107A600003290FD01AE001782A468A403A4215D0FD
:107A7000022111E0027829469140019A11420DD06D
:107A8000012109E00278294691400A463A4202D192
:107A9000019A114202D00321FFF7ACFF641CE4B24B
:107AA00030788442D3D3FEBDF8B5204B15465860DC
:107AB0000024197022469D6016E00C234B431B18CE
:107AC0001E785D68B7001F4EAD00BE1935605D7849
:107AD000AE0703D51F780126BE403243ED0703D021
:107AE0001D780123AB401C430B46491EC9B2002B35
:107AF000E3D10E48144B2146401C08F050F8F8BD65
:107B000010B50A484168002903D0407808F06AF8A7
:107B100010BD082010BD10B504484168002903D0ED
:107B2000407808F0A0F810BD082010BD24210020E6
:107B30002E2E5C68616C5C6170705F696E74706938
:107B40006E2E630000070050417A01003EB500240C
:107B500069460C70EE48019402940078002819D10F
:107B6000EC480078032815D0084600F036FC0DE0FC
:107B700001A800F051FC6B460822062104209A5E01
:107B8000595E185E08F0D5F9641CE4B268460078C6
:107B90008442EDD33EBD70B5DF4C01216078DF4DEE
:107BA000484060702968002901D0002819D0FFF7EB
:107BB000CDFF6078002814D06068401C606002F03F
:107BC000A3FFD348007800280BD1D24800780328BF
:107BD00007D008F06EFF2968002902D1C0B202F078
:107BE0003EFD70BD10B5CC4900204860CA48CC4A63
:107BF00001210C3006F015F9002801D0002010BD3D
:107C0000012010BD10B5C448012100228903C068BD
:107C100006F04EF9002801D0002010BD012010BD53
:107C200010B5BD48C06806F0ADF9002801D00020AD
:107C300010BD012010BDB84948607047B648406883
:107C40007047B54910B50822103109F069F810BD28
:107C50000146B14810B50822103009F061F810BD96
:107C6000F8B5AD481030C77804797F1CC688002C61
:107C70001CD0012C1AD06421304608F0F7FFC5B2A1
:107C800064206843301AC6B2A41C1A2060430A213B
:107C900008F0ECFFB2089219AB08D2186B00C0B222
:107CA000D21AF9B210184018801E10E0701E64211C
:107CB00008F0F2FFC5B264206843301A401EC6B215
:107CC00020460E301A214843E1E7C01D00B20028CB
:107CD000FBDB072108F0E0FF0620401A8E49C0B206
:107CE0000870F8BD8C4800787047F7B50C4682B034
:107CF00000278C4908F0BAFF0D4606463C2128466D
:107D000008F0B4FF2170E1210901284608F0AEFF18
:107D1000054608463C2108F0A9FF6070A5707D204B
:107D20000001B5B2E08010E00099002924D0642160
:107D3000304608F09BFF002901D0B0071CD0FF207F
:107D40006E30281A761C85B2E680E088FF21064650
:107D5000913108F08BFF0091002910D0642130464A
:107D600008F084FF002901D0B00708D0FF206E3052
:107D7000A842D9D900201DE0FF206F30E1E7FF20A5
:107D80006F30F5E7E088FF210646913108F06EFF7D
:107D9000002953D06421304608F068FF002901D043
:107DA000B0074BD00020217900F0A2F8281A85B244
:107DB0002079401C2071E088FF210646913108F0AF
:107DC00055FF00293CD06421304608F04FFF0029C0
:107DD00001D0B00734D00020217900F089F8A84202
:107DE000D0D9E9B2E1700498002825D04A48103073
:107DF000C278914207D121790279914203D1E18879
:107E0000C288914200D00727A1788078814201D0B2
:107E1000032007436078052108F028FF3E494A887F
:107E2000904202D04880012007438F603A480822E0
:107E30002146103008F074FF05B0F0BD0120B2E714
:107E40000120C9E734498A68002801D000208860F1
:107E500010467047F8B5044680783C214843617865
:107E6000E57840183C214843217846180427E75715
:107E700016E0E088FF219131009008F0F7FE00291C
:107E800016D06421009808F0F1FE002902D0009875
:107E900080070DD00020F9B200F02AF8401985B211
:107EA0007F1E7FB2002FE4DA7D27E4883F0114E0D3
:107EB0000120F0E7FF219131204608F0D7FE00298C
:107EC00013D06421204608F0D1FE002901D0A0077C
:107ED0000BD0FF206E30401985B2641EA4B2BC42A4
:107EE000E8D210484543A819F8BDFF206F30F2E7EB
:107EF00002461F20012907D0062901D9491EC9B20F
:107F0000C90700D01E2070471C32D0B27047000055
:107F10000E200020102000203021002028200020EA
:107F2000977B0100805101001CB5002269460A714F
:107F3000487101200090022301AA78210020FFF758
:107F4000CAFC002800D001201CBD7CB50C460546AB
:107F50004020694608710020012301AA7821009081
:107F6000FFF7B9FC0123224629460020FFF7F7FC62
:107F7000002800D001207CBD10B50446B031C8B245
:107F8000FFF7D2FF0020FFF7CFFF1020FFF7CCFF55
:107F900080212046FFF7D9FF012010BD00B5A1B018
:107FA0008021684608F0D5FE00216846FFF7E4FF0F
:107FB00001216846FFF7E0FF02216846FFF7DCFF7A
:107FC00003216846FFF7D8FF21B000BD10B5AE20F1
:107FD000FFF7AAFF0020FFF7A7FF1020FFF7A4FF7D
:107FE0000020FFF7A1FFB020FFF79EFF8120FFF7E1
:107FF0009BFFFF20FFF798FFA120FFF795FFA6202A
:10800000FFF792FFA820FFF78FFF1F20FFF78CFFDD
:10801000C820FFF789FFD320FFF786FF0020FFF776
:1080200083FFD520FFF780FF8020FFF77DFFD92059
:10803000FFF77AFF0420FFF777FFDA20FFF774FFDE
:108040000220FFF771FFDB20FFF76EFF3020FFF704
:108050006BFF8D20FFF768FF1420FFF765FFA4205A
:10806000FFF762FFFFF79AFF1E2000F04CF8012097
:108070002A498007C860012010BD10B5192000F002
:1080800042F8192000F045F80A20FEF733F80120E5
:1080900022494006C8600A20FEF72CF81E2000F096
:1080A00032F81E2000F035F8642007F0C7FC1920D4
:1080B00000F02FF8FFF78AFF10BD10B5AF20FFF7D3
:1080C00033FF642007F0BAFC1E2000F01CF81E20CD
:1080D00000F01FF812490120087010BD1048007808
:1080E000704710B5AE20FFF71FFFFFF757FF0C4991
:1080F000002008701E2000F006F8012007498007C4
:10810000C860012010BD074A03218000801801606B
:10811000704701218140014881607047000500508F
:108120004821002000070050F8B5644E306805F083
:1081300029FF634C351D607AE9790027884209D30D
:10814000604C032020601D2000F0B2F80420206065
:10815000EF71F8BD012022684107002A0ED0626845
:10816000012A0FD0227A521CD2B22272AB799A42E3
:1081700012D2606054488160298808E02060606005
:108180002772F7E71D20676000F092F869880022E7
:10819000306805F08DFEF8BD2760A98800223068A0
:1081A00005F086FE607A401C6072F8BD10B5454946
:1081B00004200860454A0021404805F032FE0028AE
:1081C00001D0002010BD012010BDF8B50C460646B8
:1081D0003F484049007809781D46174608424DD16E
:1081E00036490020091DC8713649032008601D204A
:1081F00000F05EF83148006805F0C4FE322E00D26F
:108200003226322C00D23224002F00D10127322D09
:1082100000D23225FF23710CF003F5330022C01881
:1082200051415A00002308F04BFD244EFF23361D18
:108230003080610CE003F5330022C01851415A0030
:10824000002308F03DFD7080FF23690CE803F5333F
:108250000022C01851415A00B771002308F030FDC8
:10826000B0800698F0711649002008604860886068
:108270000246301F3221006805F01AFEF8BD10B525
:108280000E48006805F07EFE0C490020091DC871EB
:108290000C4C032020601D2000F00AF80420206010
:1082A00010BD0648001DC079002800D0012070478D
:1082B000012181400448C160704700004C2100202A
:1082C000382F00207407005000050050298101005C
:1082D0000F2000200D2000201CB5202168460171D0
:1082E000472141710124022301AA32212046009432
:1082F000FFF7F1FA002838D02321684601710821E0
:108300004171022301AA322101200094FFF7E3FA10
:1083100000282AD02421684601714021417102239E
:1083200001AA322101200094FFF7D5FA00281CD0C1
:1083300025216846017100214171022301AA3221E1
:1083400001200094FFF7C7FA00280ED02E216846BE
:10835000017199214171022301AA32210120009467
:10836000FFF7B9FA002800D001201CBD10B5FFF7B7
:10837000B3FF00F00EF9012010BD1CB50F206946B7
:10838000087100200123009001AA32211846FFF74E
:10839000A2FA00280DD00120034601AA3321009043
:1083A000FFF799FA002804D068460079332801D0F5
:1083B00000201CBD01201CBD1CB520216846017198
:1083C000082141710120022301AA32210090FFF708
:1083D00082FA002800D001201CBD1CB504462F20C5
:1083E0006946087100200123009001AA3221184635
:1083F000FFF771FA00280ED00120034601AA3321AD
:108400000090FFF768FA002805D068460079C0069A
:10841000C00E207001201CBD3EB50446A820694650
:10842000087100200123009001AA32211846FFF7AD
:1084300052FA002818D00120062301AA3321009007
:10844000FFF749FA00280FD068460421415E081161
:10845000208068460621415E081160806846082138
:10846000415E0811A08001203EBD1CB5392069463F
:10847000087100200123009001AA32211846FFF75D
:108480002AFA00280ED00120034601AA33210090C9
:10849000FFF721FA002805D06846007951210840ED
:1084A00000D001201CBD1CB53A2269460A714871F2
:1084B0000120022301AA32210090FFF70CFA0028C4
:1084C00000D001201CBD1CB538246B461C71002453
:1084D0005C710123002801D068464371002905D052
:1084E000694648790421084369464871002A05D045
:1084F0006946487910210843694648710093022370
:1085000001AA32210120FFF7E6F9002800D001205E
:108510001CBD1CB520216846017147214171012411
:10852000022301AA322120460094FFF7D4F9002843
:108530000ED02E216846017199214171022301AAB2
:10854000322101200094FFF7C6F9002800D0012055
:108550001CBD1CB5202168460171272141710124F1
:10856000022301AA322120460094FFF7B4F9002823
:108570000ED02E21684601719F214171022301AA6C
:10858000322101200094FFF7A6F9002800D0012035
:108590001CBD1CB532216846017136214171012490
:1085A000022301AA322120460094FFF794F9002803
:1085B0001BD03321684601714471022301AA322184
:1085C00001200094FFF787F900280ED0302168467B
:1085D00001717F214171022301AA322101200094FF
:1085E000FFF779F9002800D001201CBDF0B5FFB0DD
:1085F000002588B02C46FFF721FB002201A9FFF7D8
:1086000074FB6846007A0C280BD26846C0791F2894
:1086100007D2684680793C2803D2684640793C28D6
:1086200004D3F5A2FA490020FDF714FE802146A8E4
:1086300008F08FFB802166A808F08BFB802106A83C
:1086400008F087FB802126A808F083FBF148C0785A
:10865000002806D0684680790C2802D90C38694673
:108660008871002003900490684643798279EAA1DA
:1086700003A808F0EDFB03A808F076FBC7B22CE0D6
:1086800003A8405D3A284DD03038C0B2132186008F
:10869000E4480091815946A80019009A08F040FB6F
:1086A000E048009A3430815966A8001908F038FB78
:1086B000DC48009A6830815906A8001908F030FBA0
:1086C000D848009A9C30815926A8001908F028FB48
:1086D000009820186D1CC4B2EDB2BD42D0D3D24870
:1086E0001EAF01685EA8013005903EAE80300137B4
:1086F00001360090002918D01F22CC49059808F0B7
:108700000FFBCA491F221F39009808F009FBC7490F
:108710001F223E39384608F003FBC4491F225D3949
:10872000304668E00A200C21B1E7662501F0DFFB46
:10873000502801D3052410E03C2801D304240CE088
:10874000282801D3032408E0142801D3022404E0DC
:10875000022801D3012400E00024B5480078002855
:1087600020D01F22B349384608F0DAFAB1491F2257
:108770001F39304608F0D4FA002626AF0FE006A8CD
:1087800040190422AC4908F0CBFAAB49781904220D
:10879000091D08F0C5FA2D1D761CEDB2F6B2A642F1
:1087A000EDD30BE0A3491F223E31384608F0B8FA5A
:1087B000A0491F221F31304608F0B2FA9F480188B5
:1087C0009F48814209D09B491F229B39059808F098
:1087D000A7FA98491F227C390CE09A4800680028C3
:1087E0000BD094491F225D39059808F099FA9149F8
:1087F0001F223E39009808F093FA002146A8FFF79F
:10880000BBFB012166A8FFF7B7FB022106A8FFF713
:10881000B3FB032126A8FFF7AFFB7FB008B0F0BD84
:10882000F8B50624884D804F884E030008F024FBDD
:10883000091C0626303C1B1B1B421B002C70FFF73B
:108840004DFC00280FD0386800280CD17148807981
:10885000002806D079487A490088884201D008204B
:1088600000E005203060F8BD2C70FFF737FC0028D1
:10887000F9D038680028F6D10220F3E72C70FFF712
:108880002DFC0028EFD038680028ECD10120E9E762
:108890002C70FFF723FC0028E5D038680028E2D0D0
:1088A000002008F091F9F8BDFFF718FC0028FAD174
:1088B0002C70F8BD2C700C20D4E7F0B5FFB000256B
:1088C00086B02C46FFF70EFAFFF7B8F9002201A98F
:1088D000FFF70BFA6846007A0C280BD26846C0797D
:1088E0001F2807D2684680793C2803D26846407921
:1088F0003C2805D3464940A2B3310020FDF7AAFC2D
:10890000802145A808F025FA802165A808F021FA01
:10891000802105A808F01DFA802125A808F019FA81
:108920000020039004906846C379027A5B1C521CB5
:1089300047A103A808F08CFA03A808F015FAC7B2FB
:108940002CE003A8405D2F283FD03038C0B213215F
:10895000860034480091815945A80019009A08F012
:10896000DFF93048009A3430815965A8001908F0C1
:10897000D7F92C48009A6830815905A8001908F0E9
:10898000CFF92848009A9C30815925A8001908F091
:10899000C7F9009820186D1CC4B2EDB2BD42D0D307
:1089A000FFF7A0F91DAB3DAC0133013400280FD017
:1089B000012816D0022853D003285AD0042862D0A8
:1089C00005286AD0062873D07EE00B200C21BFE773
:1089D0001F222249184608F0A3F920491F221F31FF
:1089E0006FE01E491F223E39184608F099F91B49CD
:1089F0001F221F3965E000002E2E5C68616C5C61EF
:108A000070705F646973705F706167652E630000EA
:108A10001405000048200020253032643A25303209
:108A20006400000058210020282000206517020063
:108A30000D200020351D02009C130200182000208C
:108A4000FFFF00002420002090200020982000201C
:108A5000253032642F25303264000000061F0200EA
:108A60001F22F849184608F05BF9F6491F221F310A
:108A700027E0F4491F223E39184608F051F9F14920
:108A80001F221F391DE0EF491F227C39184608F0CC
:108A900047F9EC491F225D3913E0EA491F22BA3930
:108AA000184608F03DF9E7491F229B3909E0FFE726
:108AB000E4491F22F839184608F032F9E1491F222B
:108AC000D939204608F02CF9002145A8FFF754FABF
:108AD000012165A8FFF750FA022105A8FFF74CFA1B
:108AE000032125A8FFF748FA7FB006B0F0BDF8B51E
:108AF00000270625D44ED54C030008F0BDF9051714
:108B000004291E2516003570FFF7E8FA00280CD05E
:108B1000CF488079002806D0CE48CF4900888842C7
:108B200001D0082000E005202060F8BD3570FFF777
:108B3000D5FA0028F9D00220F6E73570FFF7CEFA13
:108B40000028F2D12760F8BDFFF7C8FA0028FAD153
:108B50003570F7E7F0B5FFB08CB0002580210BA889
:108B600008F0F7F880212BA808F0F3F880214BA833
:108B700008F0EFF880216BA808F0EBF8684601F0E8
:108B8000F0FE002005900490B4A104A8009A08F01B
:108B90005FF904A808F0E8F8C6B2052E00D905264A
:108BA0000520801B132148431F30C4B227E004A8CE
:108BB000405D132230380006870DA948C1590BA823
:108BC000001908F0ADF8A64813223430C1592BA87B
:108BD000001908F0A5F8A24813226830C1594BA823
:108BE000001908F09DF89E4813229C30C1596BA8CB
:108BF000001908F095F813346D1CE4B2EDB2B542DB
:108C0000D5D31F2297490BA808F08AF895491F224F
:108C10001F392BA808F084F892491F223E394BA82F
:108C200008F07EF88F491F225D396BA808F078F8AC
:108C300000210BA8FFF7A0F901212BA8FFF79CF951
:108C400002214BA8FFF798F903216BA8FFF794F9CD
:108C50007FB00CB0F0BDF8B5002706247A4D7B4EEE
:108C6000030008F009F905041E0B131A12002C70FA
:108C7000FFF734FA002808D0052005E02C70FFF734
:108C80002DFA002801D003203060F8BD2C70FFF7CA
:108C900025FA0028F9D13760F8BDFFF71FFA002840
:108CA000FAD12C70F7E7F0B5FFB08EB00026802126
:108CB0000DA808F04EF880212DA808F04AF8802170
:108CC0004DA808F046F880216DA808F042F86846E3
:108CD00001F047FE0020049005905D48807801284F
:108CE00001981CD07D21C90007F0C0FF0A21019026
:108CF00007F0BCFF82B20B0013D05BA104A808F000
:108D0000A7F804A808F030F8C5B2052D00D905254C
:108D10000520401B132148431F30C4B20CE05449C6
:108D2000E2E74EA104A808F093F8EAE704A8805D02
:108D30002E2805D0761CF6B2AE42F7D300262FE0DF
:108D4000E41DE4B2FAE704A8805D2E2855D030383F
:108D5000C0B21321870042480B91C1590DA80019D8
:108D6000132207F0DDFF3E4813223430C1592DA8ED
:108D7000001907F0D5FF3A4813226830C1594DA8B1
:108D8000001907F0CDFF364813229C30C1596DA859
:108D9000001907F0C5FF0B982018761CC4B2F6B274
:108DA000AE42D0D32F491F227C310DA807F0B8FF67
:108DB0002C491F225D312DA807F0B2FF29491F223F
:108DC0003E314DA807F0ACFF26491F221F316DA888
:108DD00007F0A6FF00210DA8FFF7CEF801212DA86E
:108DE000FFF7CAF802214DA8FFF7C6F803216DA8C6
:108DF000FFF7C2F87FB00EB0F0BD0C200146A9E726
:108E0000F8B500270624104D104E030008F034F882
:108E10000504360B133212002C70FFF75FF900289F
:108E200008D0052005E02C70FFF758F9002801D084
:108E300004203060F8BD2C70FFF750F90028F9D1FC
:108E40003760F8BD8A1E0200902000209820002084
:108E50004820002018200020FFFF000025640000AB
:108E600058210020F914020025642E25640000001A
:108E700049060000FFF732F90028E2D12C70DFE745
:108E8000F0B5FFB08CB0002580210BA807F061FF82
:108E900080212BA807F05DFF80214BA807F059FF28
:108EA00080216BA807F055FF684601F05AFD0020AD
:108EB000049005900A21029807F0D8FE0246FCA112
:108EC00004A807F0C5FF04A807F04EFFC6B2052EA0
:108ED00000D905260520801B132148431F30C4B24A
:108EE00027E004A8405D132230380006870DF148C2
:108EF000C1590BA8001907F013FFEE4813223430B4
:108F0000C1592BA8001907F00BFFEA48132268305B
:108F1000C1594BA8001907F003FFE64813229C3003
:108F2000C1596BA8001907F0FBFE13346D1CE4B2A5
:108F3000EDB2B542D5D31F22DF490BA807F0F0FEF2
:108F4000DD491F221F392BA807F0EAFEDA491F224C
:108F50003E394BA807F0E4FED7491F225D396BA8C4
:108F600007F0DEFE00210BA8FFF706F801212BA871
:108F7000FFF702F802214BA8FEF7FEFF03216BA8C2
:108F8000FEF7FAFF64E6F8B500270624CB4DCC4E79
:108F9000030007F071FF05041E0B131A12002C705A
:108FA000FFF79CF8002808D0052005E02C70FFF79B
:108FB00095F8002801D002203060F8BD2C70FFF732
:108FC0008DF80028F9D13760F8BDFFF787F8002841
:108FD000FAD12C70F7E700B5FFB082B08021684667
:108FE00007F0B7FE802120A807F0B3FE802140A83B
:108FF00007F0AFFE802160A807F0ABFE0CA81F228F
:10900000B04907F08DFEAF492CA81F221F3907F089
:1090100087FEAC494CA81F223E3907F081FEA949C2
:109020006CA81F225D3907F07BFE00216846FEF721
:10903000A3FF012120A8FEF79FFF022140A8FEF711
:109040009BFF032160A8FEF797FF7FB002B000BD31
:10905000F8B50027994E9A4C0625030007F00CFF3F
:10906000050B041E2C361B003570FFF737F800285F
:1090700011D002200EE03570FFF730F800280AD03A
:1090800091488079002807D0904801889048814213
:1090900002D008202060F8BD2760F8BD3570FFF7CA
:1090A0001DF80028F9D0894801888948814201D0FB
:1090B0002560F8BD0720EDE735702760FFF70EF853
:1090C0000028F6D0012007F07FFDF8BDFFF706F875
:1090D0000028FAD13570DFE770B5FFB081B080218C
:1090E000684607F036FE802120A807F032FE802176
:1090F00040A807F02EFE802160A807F02AFE7348E2
:10910000734A01880CA82CAE4CAD6CAC914215D0C2
:109110006C491F227C3107F003FE6A4930461F224A
:109120005D3107F0FDFD674928461F223E3107F0FB
:10913000F7FD64491F2220461F3114E061491F22B8
:10914000F83107F0EDFD5F4930461F22D93107F0B5
:10915000E7FD5C4928461F22BA3107F0E1FD594975
:1091600020461F229B3107F0DBFD00216846FEF7F9
:1091700003FF012120A8FEF7FFFE022140A8FEF711
:10918000FBFE032160A8FEF7F7FE7FB001B070BDC3
:10919000F8B500270624494D494E030007F06CFE40
:1091A000050B041E25331B002C70FEF797FF0028CB
:1091B00011D002200EE02C70FEF790FF00280AD09C
:1091C00041488079002807D04048018840488142C2
:1091D00002D008203060F8BD3760F8BD2C70FEF773
:1091E0007DFF0028F9D00720F4E72C70FEF776FF0A
:1091F0000028F2D03548018835488142EDD0022060
:10920000FDF7A9F9F8BDFEF769FF0028FAD12C7027
:10921000E2E700B5FFB082B08021684607F099FD13
:10922000802120A807F095FD802140A807F091FD3E
:10923000802160A807F08DFD0CA81F22254907F0AA
:109240006FFD24492CA81F221F3907F069FD214911
:109250004CA81F223E3907F063FD1E496CA81F224F
:109260005D3907F05DFD00216846FEF785FE0121AE
:1092700020A8FEF781FE022140A8FEF77DFE032113
:1092800060A8FEF779FEE0E6F8B5002706240B4D4E
:109290000B4E030007F0F0FD052004333A42300086
:1092A0002C70FEF71BFF002826D0022023E00000D0
:1092B0002564000058210020F115020090200020B4
:1092C0009820002065170200482000201820002068
:1092D000FFFF0000D91802002C70FEF7FFFE0028E7
:1092E0000AD0FE488079002807D0FD48FD49008853
:1092F000884202D008203060F8BD3760F8BD2C707D
:10930000FEF7ECFE0028F9D00520F4E72C70FEF7FC
:10931000E5FE0028F2D0FCF7F6FFF8BDFEF7DEFE12
:109320000028FAD12C70E8E770B5FFB081B0802139
:10933000684607F00EFD802120A807F00AFD802175
:1093400040A807F006FD802160A807F002FDE44870
:10935000E44A01880CA82CAE4CAD6CAC914214D000
:109360001F22E14907F0DCFCDF4930461F221F398C
:1093700007F0D6FCDC4928461F223E3907F0D0FC16
:10938000D9491F2220465D3914E0D7491F227C317C
:1093900007F0C6FCD44930461F225D3107F0C0FCFF
:1093A000D14928461F223E3107F0BAFCCE4920465B
:1093B0001F221F3107F0B4FC00216846FEF7DCFDD8
:1093C000012120A8FEF7D8FD022140A8FEF7D4FD18
:1093D000032160A8FEF7D0FDD7E6F8B500270624E4
:1093E000C24DC34E030007F047FD050C040F0F1DCF
:1093F0000B002C70FEF772FE002801D005203060B3
:10940000F8BD2C703760F8BD2C70FEF767FE0028A1
:10941000F9D0B348B34900888842F4D00520FDF75D
:109420009AF8F8BDFEF75AFE0028EAD0F8BDF0B56C
:10943000FFB086B00025FEF701FC002201A9FEF76F
:1094400054FC6846007A0C280BD26846C0791F2865
:1094500007D2684680793C2803D2684640793C2888
:1094600004D3A44AA4490020FCF7F4FE802105A8F7
:1094700007F06FFC802125A807F06BFC802145A830
:1094800007F067FC802165A807F063FC9348C0786B
:10949000002806D0684680790C2802D90C38694625
:1094A000887100200390049068469249437982793C
:1094B000203103A807F0CCFC03A807F055FCC7B285
:1094C0001F242CE003A8405D3A2854D03038C0B2A5
:1094D0001321860089480091815905A80019009A36
:1094E00007F01EFC8548009A3430815925A80019E0
:1094F00007F016FC8148009A6830815945A8001988
:1095000007F00EFC7D48009A9C30815965A800192F
:1095100007F006FC009820186D1CC4B2EDB2BD42E5
:10952000D0D31F22764905A807F0FAFB74491F2201
:109530001F3925A807F0F4FB71491F223E3945A8C1
:1095400007F0EEFB6E491F225D3965A807F0E8FBC6
:10955000002105A8FEF710FD012125A8FEF70CFD4E
:10956000022145A8FEF708FD032165A8FEF704FDCA
:109570007FB006B0F0BD0A200C21AAE7F8B506249A
:109580005A4D604F5A4E030007F076FC0504041351
:10959000131512002C70FEF7A1FD002808D03878B2
:1095A000012801D0002000E00D20306000F0FEFD19
:1095B000F8BD2C70F8BDFEF791FD0028F9D0F8BD7C
:1095C000F0B5FFB086B00025FEF738FB002201A9F8
:1095D000FEF78BFB6846007A0C280BD26846C079F0
:1095E0001F2807D2684680793C2803D26846407914
:1095F0003C2805D340493F4A70310020FCF72AFE41
:10960000802105A807F0A5FB802125A807F0A1FB74
:10961000802145A807F09DFB802165A807F099FBF4
:109620002E48C078002806D0684680790C2802D9D8
:109630000C386946887100200390049068462D49D3
:1096400043798279203103A807F002FC03A807F0D0
:109650008BFBC7B21F242CE003A8405D3A2869D0D9
:109660003038C0B21321860024480091815905A8E2
:109670000019009A07F054FB2048009A34308159B1
:1096800025A8001907F04CFB1C48009A6830815946
:1096900045A8001907F044FB1848009A9C308159EE
:1096A00065A8001907F03CFB009820186D1CC4B297
:1096B000EDB2BD42D0D312491F227C3105A807F07C
:1096C0002FFB0F491F225D3125A807F029FB0C490C
:1096D0001F223E3145A807F023FB15E0482000205B
:1096E00018200020FFFF00005519020090200020E4
:1096F00098200020F8890100E90800005821002086
:1097000001140200102000201F22FE4965A807F066
:1097100007FB002105A8FEF72FFC012125A8FEF775
:109720002BFC022145A8FEF727FC032165A8FEF7C4
:1097300023FC1DE70A200C2195E7F8B50624F24D1D
:10974000F24FF34E030007F097FB050404131315C3
:1097500012002C70FEF7C2FC002808D038780128CF
:1097600001D0002000E00D203060FEF788FDF8BD3C
:109770002C70F8BDFEF7B2FC0028F9D0F8BDF0B5AA
:10978000FFB082B0802140A807F0E3FA802168464C
:1097900007F0DFFA802120A807F0DBFA802160A81B
:1097A00007F0D7FADB4C6846E61F6168F93EA289EC
:1097B00020AF012902D0022944D071E0114660395E
:1097C000CDB2602A0CD26021891A49101F31CDB266
:1097D0004019D14907F0A4FAA289781931461AE054
:1097E000602D00D9602547A86022CB49033007F0DF
:1097F00097FA07A860223146033007F091FAC6496C
:1098000027A82A466031033007F08AFAC14967A8C1
:109810002A46A039033007F083FA1F22BF4940A827
:1098200007F07EFABD491F221F39684607F078FA13
:10983000BA491F223E3920A807F072FAB7491F2201
:109840005D3955E0002A3ED0802A0DD28021891A48
:10985000C9050D0E4019B04907F062FAA2897819BE
:10986000314607F05DFA1BE0803A8025D4B2802CA7
:1098700000D980242A46A84940A807F051FA2A4670
:109880003146684607F04CFAA3492246803120A8A9
:1098900007F046FA9F492246803960A807F040FA4F
:1098A000002140A8FEF768FB01216846FEF764FB33
:1098B000022120A8FEF760FB032160A8FEF75CFBF5
:1098C0007FB002B0F0BD95491F227C3140A807F05F
:1098D00027FA92491F225D31684607F021FA8F4925
:1098E0001F223E3120A807F01BFA8C491F221F318E
:1098F00060A8B6E7F8B50625834E844F844C00284F
:109900000BD0012809D0022807D0042804D1FEF783
:10991000E5FB002800D13570F8BD3570FEF7DEFBA1
:109920000028F9D03878012801D0002000E00D206F
:109930002060FEF7A4FCFDF770FEF8BDF0B5FFB0A7
:1099400084B000252C46802102A807F002FA80216D
:1099500022A807F0FEF9802142A807F0FAF9802139
:1099600062A807F0F6F90020009001906C486DA104
:109970000288684607F06CFA684607F0F5F9C7B246
:1099800027E06846405D132230380006860D6748A0
:10999000815902A8001907F0C3F964481322343032
:1099A000815922A8001907F0BBF9604813226830DA
:1099B000815942A8001907F0B3F95C4813229C3082
:1099C000815962A8001907F0ABF913346D1CE4B299
:1099D000EDB2BD42D5D35648564E04786E44A0072A
:1099E0000BD51AA81F225449013007F099F95249A2
:1099F0001F221F31304607F093F9504DE0076D44A8
:109A00000BD01F224C49284607F08AF94A497AA808
:109A10001F221F31013007F083F960070AD51F228A
:109A20004549304607F07CF943491F221F3128463B
:109A300007F076F9002102A8FEF79EFA012122A87C
:109A4000FEF79AFA022142A8FEF796FA032162A8CD
:109A5000FEF792FA7FB004B0F0BDF8B500240625F9
:109A6000294E2B4F030007F007FA05040404040BEA
:109A70000A003570FEF732FB002800D03C60F8BDCC
:109A8000FEF72CFB0028FAD13570F7E700B5FFB0E0
:109A900082B08021684607F05CF9802120A807F099
:109AA00058F9802140A807F054F9802160A807F0F8
:109AB00050F90CA81F22224907F032F920492CA89E
:109AC0001F221F3907F02CF91D494CA81F223E39CF
:109AD00007F026F91A496CA81F225D3907F020F912
:109AE00000216846FEF748FA012120A8FEF744FA53
:109AF000022140A8FEF740FA032160A8FEF73CFAD5
:109B00007FB01FE0201402009020002010200020D1
:109B100098200020C42E0020C42C00206D160200C6
:109B20001A20002025303464000000005821002055
:109B300011200020E90000005C1C02006901000007
:109B40004D1A020002B000BD70B501260C25BC4CB8
:109B5000030007F091F90C07070707100F0F0F0F0D
:109B60000F0F160F2570FEF7B9FA002802D0304605
:109B7000FCF7F1FC70BDFEF7B1FA0028FAD12570B0
:109B800070BD06202070AF490020086070BD00B590
:109B9000FFB082B08021684607F0DBF8802120A862
:109BA00007F0D7F8802140A807F0D3F8802160A8FB
:109BB00007F0CFF80CA81F22A34907F0B1F8A2497B
:109BC0002CA81F221F3907F0ABF89F494CA81F2271
:109BD0003E3907F0A5F89C496CA81F225D3907F0B3
:109BE0009FF800216846FEF7C7F9012120A8FEF77B
:109BF000C3F9022140A8FEF7BFF9032160A8FEF7D0
:109C0000BBF97DE770B50C258D4C032827D00CDC03
:109C100000281BD0012812D002280FD12570FEF792
:109C20005DFA00280AD0012016E004281ED00D2875
:109C300004D10620207083490020086070BD257083
:109C4000FEF74CFA0028F9D00B2005E02570FEF74E
:109C500045FA0028F2D00A20FCF77DFC70BD257083
:109C6000FEF73CFA0028F9D00720F5E7FEF736FAB0
:109C70000028F3D1257070BD70B5FFB081B0802190
:109C8000684607F066F8802120A807F062F8802176
:109C900040A807F05EF8802160A807F05AF86B48EA
:109CA0006B4A01880CA82CAE4CAD6CAC914243D0F1
:109CB00068490978022929D063491F22F83107F041
:109CC0002FF8614930461F22D93107F029F85E4943
:109CD00028461F22BA3107F023F85B4920461F228D
:109CE0009B3107F01DF800216846FEF745F9012178
:109CF00020A8FEF741F9022140A8FEF73DF9032113
:109D000060A8FEF739F97FB001B070BD4E491F223F
:109D10007C3107F005F84C4930461F225D3106F0D2
:109D2000FFFF494928461F223E3106F0F9FF464908
:109D30001F2220461F31D4E71F22474906F0F0FFBB
:109D4000454930461F221F3906F0EAFF424928469E
:109D50001F223E3906F0E4FF3F491F2220465D39AD
:109D6000BFE770B53B490978022901D0032600E01E
:109D700004260624324D030007F07EF8050404068D
:109D8000141D05002C7070BD2C70FEF7A7F900287B
:109D9000F9D02E482E4900888842F4D03046FCF78E
:109DA000DAFB70BD2C70FEF799F90028F9D025492F
:109DB0000020086070BDFEF791F90028E2D070BD68
:109DC000F8B5821E01260C2106271D481D4C234D87
:109DD000130007F051F80B192121070A0D2B212F31
:109DE00021322100017009201EE001700A201BE0D1
:109DF00007700B2020601A48A8606868002817D0F8
:109E0000A87B00280DD113E00770FEF767F9002842
:109E10000ED020680B2801D0002609E02868002811
:109E200002D0FDF7E0FA03E0206001E0017021605C
:109E30003046F8BD01700D20F6E701700E20F3E703
:109E40009020002098200020C91A0200182000202D
:109E5000FFFF0000102000203D1C0200C42E002047
:109E6000FD2B002010B544480168002916D00021C0
:109E7000016042488068424A012180B251604B2112
:109E8000090148433F49800A48437D21090106F002
:109E9000EDFE80B200F02EF83B49087010BD70B5A1
:109EA0003A4801244460354839494160324E002522
:109EB0003560046007202ADF002803D035A2862100
:109EC000FCF7C8F9032107202BDF002803D031A2BB
:109ED0008921FCF7BFF9072026DF002803D02DA237
:109EE0008C21FCF7B7F935602548046070BD264821
:109EF000007870477D2110B54901884201D3642064
:109F000010BD294A904205D3081A052106F0C4FE67
:109F1000642108E024496439884207D3101A0521D6
:109F200006F0BAFE5021081AC0B210BD1E4AC83A47
:109F3000904205D3081A052106F0AEFE3C21F2E757
:109F40001A49884206D3101A40000F2106F0A4FED9
:109F50002821E8E7154AB43A904205D3081A0A21A5
:109F600006F09AFE1421DEE71049FA39884201D83A
:109F7000002010BD012010BD0071004000750040A0
:109F800000700040E02E00002822002000730040F6
:109F9000028000002E2E5C68616C5C6261747465E6
:109FA00072792E63000000003C0F0000DE0D0000FF
:109FB00030B593B01D461446002920D0402C1ED841
:109FC000002C1CD0030A6A461371507101A8224666
:109FD000023006F0A5FE01200090A01CC3B201AA29
:109FE000A0210220FDF777FC002806D0002D03D029
:109FF000A000201805F022FD012013B030BD002084
:10A00000FBE77CB514460D001DD0402C1BD8002C5E
:10A0100019D0020A69460A71487100200223009093
:10A0200001AAA0211846FDF756FC00280AD00120FD
:10A03000009023462A46A1210220FDF74CFC00286F
:10A0400000D001207CBD00207CBD7CB5002468468A
:10A0500004714471AA2181710125032301AAA02161
:10A0600002200095FDF737FC00281CD0052005F0E4
:10A07000E5FC684604714471022301AAA021184638
:10A080000094FDF728FC00280DD0012301AAA1218E
:10A0900002200095FDF71FFC002804D068460079D7
:10A0A000AA2801D000207CBD01207CBD10B5464906
:10A0B0000820087001464448401C06F04AFE10BDC6
:10A0C000FEB506460025FDF70DFE01218140B07862
:10A0D000CFB281018000081A7178401880B20190D7
:10A0E0003A48A9000C18607838425AD03648401CCB
:10A0F000405D002855D1207800283CD0A07881010F
:10A100008000081AE1784018019980B2884248D34B
:10A110000A31814245D30199401AC0B2092806D0BC
:10A12000062806D0032806D0002805D039E00320F1
:10A1300002E0022000E00120029023480570052083
:10A14000FDF728F902980A214843214941180A7A63
:10A150000092CB880A7949888C461D49085A614685
:10A16000FEF733F8029800281BD16078010618D456
:10A170007840607015E0B078A178884211D170788D
:10A18000E17888420DD10520FDF704F90A200090FE
:10A19000FF20FF23C330913300220146FEF715F85C
:10A1A000E3E76D1CEDB2082D9AD3FEBD10B5064C49
:10A1B0002078082802D20121621C1154FEF75FF8B2
:10A1C0000820207010BD000029220020D42E00207D
:10A1D000CC2202003A4800210170418004214160F4
:10A1E00070477CB500240425FDF77CFD01218140EA
:10A1F000CEB26846FDF725FD6846324A81780620D2
:10A20000604380180378334206D043788B4203D8EA
:10A210008078884200D92546641CE4B2032CEED332
:10A22000274842680021954202D045600170418074
:10A23000254A264B12781B68521E1A4303D004226B
:10A240004260017041807CBDF8B51D4C05466068D8
:10A25000042833D0FDF746FD0146012002468A401E
:10A260006168D2B206235943164B2678C918CB78B9
:10A27000761CB34201D2658004E06088401960809A
:10A280002078401C207008780546154216D02578A5
:10A29000AB4213D88B886488A3420FD9030601D43C
:10A2A0005040087006201923962100905B0102227D
:10A2B0000846FDF78AFF0620FDF76CF8F8BD0000A0
:10A2C00034220020F42E00200D2000202820002021
:10A2D0001CB50821FE4806F03CFDFE4C0020206025
:10A2E0006060A0601021E060601806F032FD20215F
:10A2F000F94806F02EFD6846FDF7A3FC6946C888BC
:10A300007D210901411A2046E1731030C17269466E
:10A310000979A17381726946C9786173417269468E
:10A320008978017269464978C1711CBD70B58CB0DD
:10A33000242102A806F00DFD0821E54806F009FDDC
:10A34000E44C002626606660A66010216018E66076
:10A3500006F0FFFC2021E04806F0FBFCFDF76EFC58
:10A3600001226946FDF7C1FC6946C8887D210901C3
:10A37000411A2046E1731030C17269460979A17310
:10A3800081726946C9786173417269468978017240
:10A3900069464978C171CE4D01200E3DA870042256
:10A3A00002A910206E60FFF72CFE002810D068462E
:10A3B000007AD6280BD1032102A800F084FB69465D
:10A3C000C97A814221D16846007AD62802D001207C
:10A3D0000CB070BD6946C148497A01706946897AF6
:10A3E0004170082202A92020FFF70BFE0028EFD0C1
:10A3F000072102A800F067FB6946C97B814204D1AE
:10A40000072202A9B64806F08BFC052202A93020DB
:10A41000FFF7F7FD0028DBD0042102A800F053FB72
:10A420006946097B81420AD1029E3046FDF703FC52
:10A43000012269463046FDF758FCFDF711FC212248
:10A4400002A94020FFF7DDFD0028C1D0202102A88D
:10A4500000F039FB08A9097A814204D1202202A91F
:10A460009D4806F05DFC072202A97020FFF7C9FD98
:10A470000028ADD0062102A800F025FB6946897BA3
:10A48000814204D1062202A9964806F049FC09221D
:10A4900002A98020FFF7B5FD002899D0082102A865
:10A4A00000F011FB6946097C814204D1082202A90F
:10A4B000874806F035FC0D2202A9B020FFF7A1FD68
:10A4C000002885D083480D2202A9103006F028FC10
:10A4D000102202A99020FFF794FD002887D002A83F
:10A4E0000FC80FC4686072E700B589B024216846C0
:10A4F00006F02FFC07227A49684606F011FC072176
:10A50000684600F0E0FA6946C8710123082220205D
:10A51000FFF74EFD002877D0FDF790FB0090042157
:10A52000684600F0D0FA6946087101230522302000
:10A53000FFF73EFD002867D020226749684606F0F5
:10A54000EFFB2021684600F0BEFA08A9087001233D
:10A55000212269464020FFF72BFD002854D0062217
:10A560006049684606F0DCFB0621684600F0ABFA5D
:10A5700069468871012307227020FFF719FD002822
:10A5800042D008225249684606F0CAFB08216846B4
:10A5900000F099FA69460872012309228020FFF72A
:10A5A00007FD002830D04B490D221031684606F0D7
:10A5B000B7FB01230D226946B020FFF7F9FC002804
:10A5C00022D0444B0FCB03936B4607C301231022C9
:10A5D00069469020FFF7ECFC002815D0D62069468C
:10A5E00008703E4802784A704078887003216846B7
:10A5F00000F069FA6946C870012304221020FFF7B1
:10A60000D7FC002800D0012009B000BD38B53A20A1
:10A6100069460870012401231A4669460020FFF7A5
:10A62000C7FC2146641CE4B20A2902D20028F2D0F9
:10A6300001E0002812D00124012269460020FFF722
:10A64000E0FC002803D0694609783A2906D0214663
:10A65000641CE4B20A2901D20028EDD038BDFEB551
:10A6600004461C481F4D0168002628883746814251
:10A670000BD20919814208D303204B23DB00009041
:10A68000581002220146FDF7A0FD17480168114845
:10A690001030002904D01549048009780173FEBDEB
:10A6A000052C01D3052300E0234609490E39002C6F
:10A6B0000CD0AA780D460835EB5C5A436243960AE3
:10A6C0000B786208D718E207D20F0A7002880FE0F1
:10A6D0004A220020442F0020D42E00201C200020DD
:10A6E0004820002088200020282000202C20002046
:10A6F000121902804288FA4D921942808288D2193A
:10A7000082802868001928606A6892196A60AA68BD
:10A710000E46D219AA604968884201D9401A00E061
:10A72000081A80B20A28BAD9EE4F386802F066FAE1
:10A73000002821D00A21686806F098FA04460A2108
:10A74000A86806F093FA01460722684602702A6854
:10A750004270130A8370120CC2700471220A427193
:10A76000220C8271C1710A0A0272090C41720146FF
:10A770000A22386802F044FA0021012000F00CFEA1
:10A7800028687060FEBDF0B5D54C87B010342088C5
:10A79000FFF75AFDE27AD44E0A2A52D920880028BF
:10A7A00005D1217B002902D17178002949D00027E9
:10A7B0000297039704970597E37969464B72237ACA
:10A7C0008B72637ACB72A37A0B734A73227B8A7380
:10A7D000C873000A087460884874000A8874A088E6
:10A7E000C874000A087502A80C21013000F06BF94A
:10A7F000BD4DA071694608720E3528880123FF30CF
:10A80000FF30023080B20D2202A9FFF7D1FB0028F1
:10A8100017D028883F2110304902884201D32F8069
:10A8200002E028881030288068882A88904208D161
:10A8300068881030884201D36F8002E06888103049
:10A8400068800120B0700021022000F0A5FDA4481E
:10A850000D21103006F07DFA6846FDF7F2F96846E2
:10A860004078E0716846807820726846C0786072EF
:10A8700068460079A0726846C0887D210901401AA7
:10A88000E072207B707099480078207307B0F0BDAB
:10A8900070B5934D0026E87B88B00A2846D96A7BBC
:10A8A00069464A70AA7B8A70C87028680871020AD3
:10A8B0004A71020C8A71000EC87168680872020A37
:10A8C0004A72020C8A72000EC872A8680873020AE3
:10A8D0004A73020C8A73000EC87300A80F2101305E
:10A8E00000F0F1F8804C2873694608700E34A079A6
:10A8F0000123FF3001301022FFF75AFB002815D04A
:10A90000A0791030702801D3A67102E0A079103030
:10A91000A071E079A179884208D1E07910307028DF
:10A9200001D3E67102E0E0791030E07100210120EE
:10A9300000F032FD2E606E60AE6004A8EE60FDF7A0
:10A9400080F96846C07C68736846007DA8736846D5
:10A95000C08A7D210901401AE8736348466008B047
:10A9600070BD10B55E4B04460FCB0FC4103CFF20EA
:10A970006073A073E07320460F210D3000F0A3F840
:10A98000207310BD70B5584D04460E35688829886F
:10A990000026884224D10D21204606F0DAF9FF2056
:10A9A0006070A070E070207160714D481030017BC4
:10A9B000A1710178E1710188090A217281786172BF
:10A9C0004188090AA1720179E17280880C21000A8C
:10A9D0002073601C00F077F82070434886701BE0FD
:10A9E00068880D22FF30FF30023080B22146FFF729
:10A9F00008FB002807D068883F21103049028842B0
:10AA000007D36E8008E00D21204606F0A2F9002051
:10AA100070BD688810306880012070BD70B5324C00
:10AA200005460E34E079A179884212D110212846DA
:10AA300006F08FF9FF206870A870E8700C22284992
:10AA4000281D06F06DF90F21681C00F03CF82870F5
:10AA500017E0E0791022FF3001302946FFF7D1FAE4
:10AA6000002805D0E0791030702807D3002007E0D7
:10AA70001021284606F06DF9002070BDE0791030F5
:10AA8000E071012070BD18480E3041880088814275
:10AA900003D115488078002800D001207047124863
:10AAA0000E30C1798079814201D0012070470020A9
:10AAB00070470D480E308188491C818070470A48D4
:10AAC0000E308088704710B503460022104603E020
:10AAD0009C5C6040521CD2B28A42F9D310BD000087
:10AAE000442F0020D42200203C22002028200020D7
:10AAF00007480121C16005221204426082680A43AE
:10AB00008260044801607047044903480860704748
:10AB100000050140000001403546526E000601402C
:10AB2000FEB5064601200290FFF7EEFFFE4DFD49FF
:10AB3000E81DF930C51DF935012E07D0022E05D0CC
:10AB4000032E0DD0042E0BD00020FEBDF54A121F9F
:10AB5000541DD27857180021A981F349019109E0C9
:10AB6000F04A121F141DD2785718A989EE4A8A1884
:10AB70000818019200904AE02078002805D00128AA
:10AB80001DD000200290A88155E0A889FF2108303F
:10AB9000013188423DD8641CA881082221460198D1
:10ABA00006F0BEF8083408222146009806F0B8F8EE
:10ABB000019808340830019000980830DAE7A88935
:10ABC000782810D10821019806F0C3F808210098D0
:10ABD00006F0BFF8A8890830A881019808300190D4
:10ABE000009808300090A889FF2110300131884278
:10ABF0000FD8641CA88110222146019806F090F815
:10AC0000103410222146009806F08AF81034BC4215
:10AC1000B2D3012E01D0042E0DD1C248001F0079FD
:10AC20006860012028600020A873C04802680121E4
:10AC300009040A4302600298FEBDBD490020486035
:10AC40000870BC49086088607047F8B500260C465B
:10AC5000002959D0B34FB64D3F1F6A68002A06D06D
:10AC6000012A1CD0022A22D0032A15D132E002295F
:10AC70000FD9437802781B02D218AF4B92B29A4296
:10AC800007D101226A600022A41E2A70A4B2801C8F
:10AC900002E0641EA4B2401C002CDED134E0027835
:10ACA000BA700222401C641EA4B26A60F4E7027803
:10ACB000FA70002A01D0802A02D90126002200E081
:10ACC0000322641EA4B2401C6A60002C1CD0002E1B
:10ACD000C3D019E02978FB7862189A420AD35A1A2D
:10ACE0007B181B1D0146184606F01AF801260020A5
:10ACF000686009E07B181B1D01462246184606F0D5
:10AD00000FF82878001928703046F8BDF1B585484D
:10AD10000024001FC2788CB0802A18D88078089050
:10AD2000070703093F0F002B12D07E48001F8179CF
:10AD30000391C679017A457A009545790079012B0E
:10AD40003AD0022B7ED0032B7DD0042B7CD0DFE1C8
:10AD50003B0006F091F806041B2227C52CC5FFF71F
:10AD6000AEFE73490831488209A871DF704809A90D
:10AD700006220131143005F0D3FF6D491A22083143
:10AD8000684605F0CDFF01241A2254E1FFF7AFF821
:10AD900069460124087022464EE164480124016896
:10ADA00006226EE16148012401680A2269E15F48D8
:10ADB00001240168202264E13B0006F05DF80A06E8
:10ADC000304F5D6175799296E591062ABFD17D225B
:10ADD00012018218684642810B2D00D90B2505729D
:10ADE00003981E2800D91E206A46D071172E00D95C
:10ADF0001726104696713B2900D93B2141710098D6
:10AE00003B2800D93B20107101A8FDF723F8FCF77F
:10AE100012FF002004900C98016904A85EE0FCF782
:10AE20000DFF00226946FCF760FF6846C1887D205F
:10AE30000001091A6846017201794172C178817274
:10AE4000817802E0A4E0FBE01EE1C1724178017369
:10AE5000017841730124062202A9EDE0022A3FD3C2
:10AE600036490A78904200D008704878854200D070
:10AE70004D70FFF71EFE32E0012402222F49DBE075
:10AE8000052AA3D108282BD22D4A800015548018FA
:10AE9000039B43708670C170FFF70BFE012000908A
:10AEA0000C980169684619E0012420222449C3E076
:10AEB000072A8BD10328E6D206225043214A155493
:10AEC0008018039B43708670C17000998180FFF7E2
:10AED000F0FD022001900C98016901A88847012427
:10AEE00016E1012412221749A6E00124FFF7E1FD33
:10AEF0000C4D154E2D1FE878022830D33178287973
:10AF0000814209D0002800D0012030700320009039
:10AF10000C980169684688477178687981421ED02B
:10AF2000002813E0682F0020C42C002020200020DF
:10AF300054220020C42E002021FF00001C200020ED
:10AF4000D42E0020F42E00204820002000D0012024
:10AF50007070042000900C98016968468847E87872
:10AF6000032804D3A979002900D00121B170042855
:10AF700009D3E979F170052805D3297A31710628BA
:10AF800001D3687A7071C3E001240722624953E05B
:10AF90003B0005F071FF080518292C3033393EBD00
:10AFA000062A0FD15D4A9070D5700398002800D012
:10AFB00001201071567100980124000208181080B9
:10AFC000FFF777FDA4E05548694682780A70C27899
:10AFD0004A7002798A704279CA7000880871000A42
:10AFE00001244871062227E0FFF772F977E7012470
:10AFF0002146204605E00124204607E001242146A1
:10B00000022000F0C9F983E00124022000F0FFF9DA
:10B010007EE0012404A8FFF7A4FC6846017F0170CC
:10B02000417F4170817F8170C17FC17004A807C8D2
:10B0300001AB07C310226946089800F075F967E074
:10B04000012F06D0022F04D0032F05D0042F03D0E8
:10B050005EE03349FF2D04D03846FFF761FD04461A
:10B0600056E0304B01241C6058602F489C73921EA0
:10B070000270401C8922891D05F052FE2B48016890
:10B0800022041143016043E0002F02D0012F26D09B
:10B090003EE0234D012A3BD1254E0124317803297E
:10B0A00006D0032808D001290AD001280CD00EE0D0
:10B0B000032811D0002000E00120FBF734FA06E05D
:10B0C000012809D00B2000E00A20FCF763F9287959
:10B0D000042801D3002000E02879307018E0104FD8
:10B0E000092A13D3002811D00398BB7A009A0002D2
:10B0F0001B022818D218090293B27118FA7A3D7B04
:10B1000080B289B20095FDF760F801E0FDF7B7F86D
:10B1100020460DB0F0BD000048200020882000200F
:10B12000642F0020C42E0020FC2B002020200020B3
:10B1300010200020F7B582B004980026001D009072
:10B14000C0B201271421401E05F0A6FDB24C401CE0
:10B150002178C5B2607881422178607801D9081AD7
:10B1600001E0081A0930A84241DA002005B0F0BD1C
:10B17000607815214843A9494018002F19D0222191
:10B180004170FF2181700299C170002704990171FB
:10B19000002D08D014210170401D1022039905F0E4
:10B1A000BFFD10261BE000990170401D049A039911
:10B1B00013E0002D0AD0142101700399401C891955
:10B1C000142205F0ADFD1436F6B208E00499891B8F
:10B1D000CAB202700399401C891905F0A1FD60787C
:10B1E000401CC0B260700A2801D30020607028465D
:10B1F0006D1EEDB20028BBD10120B7E730B587B096
:10B2000004A87BDF844CE06802F0BCFE2078617803
:10B210007D25ED0088421ED1606800286AD0C007F5
:10B2200008D0FFF73CFC002838D103E01022694623
:10B2300023200EE0207980072DD5FFF724FC00287D
:10B2400029D06846FFF79EFB002834D00D226946BE
:10B250002520FFF76FFF2078152148436F494118DB
:10B260000A78491CA06801F092FB002823D02078BE
:10B27000401CC0B220700A2801D300202070207822
:10B280006178884217D12079C0070DD0FFF707FCFD
:10B29000002810D108E02079C0072BD06846FFF7BE
:10B2A000BDFB0028C2D106E02079800719D5FFF741
:10B2B000EAFB002815D06846008A5949FF23484315
:10B2C000400AC117420CC903C003F5331143C0182B
:10B2D000002251412A46002305F0F2FC00220146DB
:10B2E00005E02079C00705D000220F214904E0685D
:10B2F00002F0DEFD07B030BD10B547498860002080
:10B3000048700870486001464348464A0C3002F0D5
:10B3100088FD10BD10B540480021417001704160AA
:10B32000C06802F02FFE10BDF7B582B001271546A8
:10B330000E46FF0368467BDF01F049FA002813D070
:10B34000684600883649FF234843400AC117420C2B
:10B35000C9031143C003F5330022C01851415A00FC
:10B36000002305F0ADFC07462B4CA06801F00DFB57
:10B37000002810D020786178884207D1E06802F078
:10B3800001FE00223946E06802F092FD2A4631466D
:10B390000298FFF7CFFEE9E6FEB5064601250F4607
:10B3A000ED0368467BDF01F012FA002813D06846EF
:10B3B00000881B49FF234843400AC117420CC903B8
:10B3C0001143C003F5330022C01851415A00002335
:10B3D00005F076FC0546104CA06801F0D6FA00286E
:10B3E0000DD06068002F0BD0304360600AE0E06849
:10B3F00002F0C8FD00222946E06802F059FDFEBDBA
:10B400003042FCD0207861788842F0D0FEBD0249FD
:10B410004A6882434A60704778220020E82F002063
:10B42000E2040000FDB10100F0B5FB4D0C462978A7
:10B430008BB01646002921D1032269460A71020CFD
:10B440004A71020A8A71C871201D009002AB042261
:10B4500001A9002004F0CBF907000AD1201DFAF75A
:10B4600059FE2878002809D0224603A9304605F065
:10B4700057FC0020287038460BB0F0BD1120FBE7C8
:10B48000012801D1E4490870704710B50A46002828
:10B4900050D0002A4ED003461121203BC9015F2B1A
:10B4A00003D800014318102109E027235B02DB4C7D
:10B4B000C31AA3420DD8DA49400143182021002BBA
:10B4C0003AD01170521C1846FFF7AEFF002833D156
:10B4D00030E0D44BC3185D2B04D8FF232133C018B0
:10B4E00080B2DEE703210903884202D11523DB0184
:10B4F00004E0CD49884203D139239B011021E0E7C4
:10B50000C949491C884202D15B235B01F6E7C64961
:10B510003123C91D9B018842F0D04C1C6321490195
:10B52000A04205D0641CA042E8D0631C984203D11D
:10B530000B46E3E7012010BD002010BD38B50C46D6
:10B54000BAA1096800910146B94AA0394300914265
:10B5500002D8FF3B413B2DE0B649B74A4118914222
:10B5600001D8B64825E00321B14A0903411A243223
:10B57000914201D8B2481CE02721A84A4902411A49
:10B58000521E914201D8AF4813E0A649D13141186B
:10B590003B2901D8AC480CE0A24941185D2901D8EB
:10B5A000AA4806E09F49DF394018052835D8A64843
:10B5B0006E381B18002B30D020202070A4486A461B
:10B5C00002211818FFF730FF002826D168460078BE
:10B5D000002803D16946497800291ED069460246F1
:10B5E0004978A13A082A07D8A12905D35E20424309
:10B5F00050184001974909E0B03847280DD8A129D3
:10B600000BD35E2250434018934940014018621CFE
:10B610002021FFF709FF002801D0002038BD0120BC
:10B6200038BD38B50C4681A1096800910146A239A0
:10B630004300552902D8FF3B413B2BE08749FF22BD
:10B6400041180332914201D8854822E079497A4A6B
:10B65000C91E4118D21E914201D8824819E0032127
:10B66000734A0903411A2432914201D87E4810E0FE
:10B6700027216A4A4902411A0A3A914201D87B4875
:10B6800007E06849D1314018FF21CE31884242D8C5
:10B6900077481B18002B3ED02020207075486A4642
:10B6A00002211818FFF7C0FE002834D1684601783F
:10B6B000002902D1407800282DD068464078A4396E
:10B6C000222928D80246403A3E2A04D89D225143D6
:10B6D0000818403807E00246A13A5D2A1BD89D228F
:10B6E0005143081862386449400040186A460221F4
:10B6F000FFF79AFE00280ED168460078621C01020E
:10B700006846407808185D49400140182021FFF73D
:10B710008BFE002801D0002038BD012038BD38B58F
:10B720000C460021009103463B21A13B09018B42BD
:10B730002CD94049CB22491F4118D200914201D84F
:10B740004F4922E003213A4A0903411A2C3291421F
:10B7500001D84C4919E02721304A4902411A0A3AD6
:10B76000914201D8484910E02B218902474A411AE9
:10B77000914202D83249453907E0F9212E4A09029F
:10B78000411ACD32914238D841494318002B34D068
:10B79000202020703F49580045186A46022128465B
:10B7A000FFF742FE002828D168460378002B02D11B
:10B7B0004078002821D01846A1380F2809D26946C0
:10B7C0004978A12905D35E225043401840013249EF
:10B7D0000BE0B03B182B09D868464078A12805D368
:10B7E0005E214B4318182D4940014518621C202149
:10B7F0002846FFF719FE002801D0002038BD01209F
:10B8000038BD10B5044900200870254903F02CFF0D
:10B81000002847D0002010BD88220020A65100003B
:10B8200020610000FF00FFFF0130000000000A005F
:10B83000B1030000F0DFFFFF3206000044C7FFFF46
:10B84000CAB3FFFF767FFFFF62C2FEFF38C1FEFF73
:10B850009EBA0C0060FC00002066010039FDFFFF6D
:10B8600036FBFFFFAAC2FFFF6AAFFFFF327BFFFF7D
:10B870004CBEFEFF203C1100FE480E00801001006F
:10B880009CE3FFFF0ADAFFFFE8BFFFFF9D2B0000EC
:10B890002392FFFF40920B0040B70500A042060034
:10B8A000F4220200EE49002005F046FD0120B2E737
:10B8B00010B5002003F060FFEA4904200860091F6A
:10B8C0000860E849083108600320091F086001206A
:10B8D000E549C00488609EE718B50022009202780E
:10B8E000401C6B461A70802A02D20A80012018BDC3
:10B8F00004785C701346401CC03B202B07D2D00656
:10B90000A206400D920E80180880022018BD037810
:10B91000684683701046E03810280AD29001A206CB
:10B92000920E80189A068001920E801808800320DB
:10B9300018BD002018BDF8B50746002014460E4675
:10B940001070FFF7E1F82121304605F002FAC74DEB
:10B950006878002805D131463846FFF796FD002863
:10B9600020D16878012828D13146384600F065F8A2
:10B97000002817D131463846FFF753FE002811D171
:10B9800031463846FFF7DAFD00280BD131463846FC
:10B9900000F0B8F8002805D131463846FFF7BFFE61
:10B9A000002801D00120F8BD3146384600F003F9E7
:10B9B000002802D001202070F4E70020F8BD10B567
:10B9C000ABA09EB000681D9000246846048024212E
:10B9D00002A805F0BEF9684604712422A5A10BA8AF
:10B9E00005F09EF969461DA8FFF776FFFFF709FFEE
:10B9F00000281ED0684601AA02A90088FFF79BFF15
:10BA0000002816D021220BA902A805F0B4F9974905
:10BA1000002810D0012048709F4C242114A805F064
:10BA200098F901AA14A92046FFF785FFFFF740FF08
:10BA300001201EB0EFE64C70EEE7024610B5203A4A
:10BA400003015F2A02D85B2080014BE00246A03A46
:10BA5000DF2A02D85320800144E00246FF3AA13A8F
:10BA60002F2A02D84B2080013CE00246FF3AF13AEF
:10BA70000F2A02D84320800134E021221201821AC9
:10BA80000F2A02D83F2080012CE0F5225201821AB1
:10BA90005F2A01D8814825E037221201821A5F2AE5
:10BAA00001D8C0331FE001229202821A5F2A02D815
:10BAB000092080010EE049221201821A6F2A02D861
:10BAC0001520800106E059221201821A6F2A03D83C
:10BAD000392080011B1A06E007225202801A5F28D3
:10BAE0000CD86F481B18002B08D0102008704A1C77
:10BAF00001461846FFF798FC002801D000208AE68E
:10BB0000012088E638B50C460021009162490346C1
:10BB1000203BE0318B4227D301214903614A411A7E
:10BB2000914203D2C1214901431A1DE003210903B7
:10BB3000411AFF2901D25C4915E019214902421A34
:10BB40005A498A4201D25A490DE027225202594BE2
:10BB5000821A9A4201D2584905E07F225202821A83
:10BB60008A4224D255494318002B20D0202020702F
:10BB70005349580040186A460221FFF755FC002837
:10BB800015D168460078002803D169464978002914
:10BB90000DD05E21484369464978621C40184949E6
:10BBA000400140182021FFF73FFC002801D0002071
:10BBB00038BD012038BD30B589B00C4600216A4639
:10BBC000117003214902431A42014100FF2B04D89E
:10BBD0003D48101840183D4910E03D4BC318AF2BAD
:10BBE00004D83C48101840183B4907E03B4BC018AC
:10BBF0008F2819D83A48101840183A49451813D0D8
:10BC00006A4601212846FFF70FFC00280CD1684640
:10BC10000078002808D0102806D201AA2021681C2C
:10BC2000FFF702FC002802D0002009B030BD6846B2
:10BC3000007801A94000207068460078641C401E0E
:10BC400040B209E00A5C22706B460A181B78127C2D
:10BC5000E254641C401E40B20028F3DA0120E4E7FD
:10BC600081B40100480700500005005088220020E0
:10BC7000E383A00020101010FF1090040404FC8245
:10BC800082838280000444827F01000101013F40E1
:10BC90004040407800000000FF060000C047FEFF63
:10BCA000C071FFFFFF070000E0DFFFFFFF010000A2
:10BCB000E0DEFFFFFF510000E0C4FFFFE066FFFF92
:10BCC0003E7B0D00607C07000040FFFF01B80000D4
:10BCD000B004FFFF00B6E0FF61CFFEFF9001FFFF61
:10BCE0000068E0FF81CAFEFF10B54348434C00786E
:10BCF0002188401E084212D041486168415C002002
:10BD000000F014F960686421401C04F0AFFF61602A
:10BD100020883C49884201D0401E208010BDA06888
:10BD200002F030F900200146606000F0FFF80020CA
:10BD300000F028F934490C20086010BD10B53249D4
:10BD40000C2008602D48314A0121083002F069F8C2
:10BD5000002801D0002010BD012010BD7FB5284B68
:10BD60000C46054664330FCB6E460FC6224800785A
:10BD700000282AD126480078002803D125480078D9
:10BD8000002822D1012069464873087016204870A7
:10BD9000684600F04BF8012000F0F4F8174E002C34
:10BDA00014D0641E642044433480FF23690CE803EC
:10BDB000F5330022C01851415A00002304F080FFDF
:10BDC00001460022B06802F073F87FBD0020C04336
:10BDD0003080EAE710B5094CA06802F0D3F80020E3
:10BDE0000146606000F0A2F8002000F0CBF80649A0
:10BDF0000C20086010BD00000E2000208C220020C6
:10BE000010230200FFFF000058070050E9BC0100AA
:10BE1000482000200D20002010B50446102804D230
:10BE2000E0B247DF0120A04045DF10BDF8B5044671
:10BE30000078401E032824D2677B092064269F498E
:10BE400003259F4A3B0005F017F8060406090F1664
:10BE5000181C086109E00861FF2003E00620086162
:10BE60007D20C000906001E00D619660944A2078CA
:10BE7000106100221CE00120EDE700200861402055
:10BE8000F0E70020C043F8BDA3185E789C468D4DB6
:10BE90009300EE50B7008C4E0325BE193560894ED5
:10BEA00000250C36F55063469D7A854B9D54521CF7
:10BEB0008242E9D385480122C26000228A6080481C
:10BEC0007E4D83684035C360EB604A60804B08213B
:10BED00019607F4EC03EF260B260726032601546FB
:10BEE00016E07748405D81007A480A18A800811959
:10BEF000680007193879FFF78FFF7148405D8100AE
:10BF000074480A1872497879B439FFF785FF6D1CB7
:10BF10006B4800698542E4D303210A202BDF0A2005
:10BF200026DF6A49012008600020F8BD654A8000CC
:10BF30000C3A115066490020C039C860644966480F
:10BF4000086066484168614A0B030121002B02DB4F
:10BF50005160CB044360116070475949C8605C4927
:10BF60000020C039C8605A495B4808605B48416896
:10BF7000564A0B030121002B02DB5160CB044360C6
:10BF800011607047F8B50121504A002804D0534B86
:10BF9000C80458601160F8BD516000242746484E1F
:10BFA00010E047484E49005D82004E48101801617C
:10BFB0004448A5004059012100F077F841480C3071
:10BFC0004751641C30698442EBD3F8BDF8B5404852
:10BFD0000025C038C5604149681E8860384C374E1E
:10BFE000E0684036A060F0603E4F656052E0354A40
:10BFF00088000C3A1258002A13D0A3689A421AD328
:10C000002F4A515C364A8900C9190A612D490858DE
:10C01000012100F04AF8606881002A480C30455040
:10C0200035E0274A515C2E4A8900C9190A61254921
:10C0300008580021EDE783191A60224A0C32125881
:10C04000002A24D11E4A535C1E49012209588C46FD
:10C050008A4025498A609B00D919244A8E460A6184
:10C0600000BF00BF00BF012219461A4BCB181A604F
:10C0700061460A02D21C13231B041A4371460A614B
:10C0800000BF00BF00BF01210E4A0C321150606892
:10C09000401C6060616820698142A8D30C49082077
:10C0A00008600A4901200860F8BD012282400E485C
:10C0B000002901D082607047C260704700A500402F
:10C0C00098220020C83000200007005000A0004047
:10C0D00000A20040006000400808000000A30040EB
:10C0E000001F03000065004000050050031F010011
:10C0F00010B5FE4C6168A068884210D02C21FC4A23
:10C10000484381184B68012B0AD01C31105A97DF25
:10C11000002804D1207A401C4007400FA06010BDC9
:10C12000105A0989002295DFF2E710B5EF4C07217C
:10C13000E160F049097801290BD12178022908D260
:10C1400002460521C903E06901F0B2FE2078401CD7
:10C15000207010BD38B50446012168468170E64A5A
:10C160000280227B827020896A4690DF010003D022
:10C170002046FFF7DAFF38BDDC490220C86038BD31
:10C18000DC490978012904D1D849C968052900D0BA
:10C19000E0E7704738B50446D848018CFF2903D042
:10C1A000818DFF2908D014E0C08B6946401C0880AF
:10C1B0004880208993DF06E0408D6946401C088056
:10C1C0004880208993DF010003D02046FFF7ADFFB0
:10C1D00038BDC6490420C86038BDFEB50E46C988C2
:10C1E00007460846FF380B3801D009300FD1C34845
:10C1F000C18B002909D0418A002906D0408D002832
:10C2000003D03846FFF7C6FFFEBD052101E0002937
:10C2100003D03846FFF789FFFEBDB8480024014629
:10C220000A3102910C31223025460191009016E02E
:10C230000A20684384190E342188B148091809D0AE
:10C24000B048081818D0AE49C91C401806D121467C
:10C25000029801E02146019800F0DFFA6D1CB089D8
:10C26000A842E5D8002C0AD020896946401C0880E5
:10C27000A2480089488004E021460098ECE79F49E5
:10C28000891D384600F0ADFAFEBDF7B5984D002483
:10C290001646964FC43D54E03869030004F0ECFDA7
:10C2A00009060B10151A1E23283650000198005D50
:10C2B0002872012043E00198005D687202203EE090
:10C2C0000198005DA872032039E00198005DE872D2
:10C2D000042034E00198005D28732FE00198005D90
:10C2E000687306202BE00198005DE881072026E0B6
:10C2F0000199E889095D09020843E881082038614D
:10C300007B48B43878610020788019E00198015D9D
:10C3100078690170401C78617988491C89B27980FC
:10C32000EA898A420CD100210170401C7861042006
:10C330002860009801686E48C43888470520386135
:10C34000641CB442A8DBFEBDF8B51646674A074632
:10C35000D0681D46052801D00820F8BD50682C2360
:10C360004343401C4007400F5060614C63481C1918
:10C37000408AE08320460830606200202084012249
:10C380002277207220460422093004F0C9FC0520DF
:10C3900011E02978221811726988401C002907D001
:10C3A000221811726988401C090A22181172401C57
:10C3B0002D1D761EF6B2002EEBD1608438892080C8
:10C3C00002206060FFF794FE0020F8BDF0B504463F
:10C3D0000C318888B5B0002830D0484A0D88D38BFE
:10C3E0001046408D9D4204D1167E6D46AE71D28AB4
:10C3F00007E0854222D1414D20352E796D46AE7140
:10C40000528CAA800A889A424ED18A792A72CB79B4
:10C410006B720B7A2846AB724D7AC5724D89858155
:10C4200089890327C1810097002A09D0022A05D1F2
:10C43000012B03D1FBF723FFFFF7CCFC35B0F0BD98
:10C44000216888476846807A002501221223274EFA
:10C4500003A901281AD00428F0D16846407A0028A0
:10C4600001D01028EAD130A80271C3800772B4222B
:10C47000428131AB02222046FFF766FF002803D03D
:10C4800021A22749F9F7E6FE3561D7E730A8027106
:10C49000C38031AB01222046FFF756FF0028F3D0BE
:10C4A0001F4919A20D39EDE78242C7D18A88891D3B
:10C4B0002046FFF7EAFEC1E770B505460B4C0020A9
:10C4C000A0600121E16060602070E06901F05AFD28
:10C4D0000A4E3078FE2803D1A87AFF2828D0307081
:10C4E000C0B2042824D22E2148431BE0AC220020F5
:10C4F000A43100201C20002031F40000BC330020B7
:10C50000F3EDFFFF244BFFFF2E2E5C7365727669FF
:10C5100063655C626C655F616E63735F632E63006D
:10C52000F7020000A1692E224018DF4904F0F8FB51
:10C530002E21DD4804F00DFCFF2030700021E87250
:10C54000C9432981A87270BD1278112A01D0142A1A
:10C5500001D189788172704770B5D44A0C88D66849
:10C56000FF22D14D330004F087FC0715051E383D2E
:10C57000420A1900102C0DD18988018107E0172C7F
:10C5800001D0142C0AD16988C94B994203D02A7072
:10C59000FFF7E0FD70BD00F032F970BD112CFCD149
:10C5A000FFF78AFF70BD302CF8D10A46C9880029F0
:10C5B00002D0FFF7BAFD70BD117C2971D189698065
:10C5C0009189002907D0518AE980918A2981A91D82
:10C5D00000F007F970BDD188EBE7322CDED1FFF710
:10C5E000FCFD70BD332CD9D100F024F970BD382C7E
:10C5F0000CD0372CD2D1C888002804D00022114694
:10C600000420FEF791FEFFF773FD70BDFFF7DEFE1D
:10C6100070BD10B5100003D0A64AA749F9F71AFE5D
:10C6200010BD7FB5044608680E46002867D0214635
:10C630000C31A24863DF002804D09F499D4A0F3186
:10C64000F9F708FE01AD9D48A91C103063DF0028F2
:10C6500004D09949974A1231F9F7FCFD9748A91C73
:10C66000203063DF002804D0F121924A8900F9F7D5
:10C67000F1FD9248A91C303063DF002804D08E49B8
:10C680008C4A1831F9F7E6FD306820607068606008
:10C69000FF250026A572E672701E20812E21824899
:10C6A00004F057FB8648814C466486647E486946A0
:10C6B00005700120E060C881B8208881814821464A
:10C6C0000290203102A800F02BFD002804D0F721B1
:10C6D000784A8900F9F7BEFD73487B4AB838A061F3
:10C6E000724800211C3001F09CFB040004D0724908
:10C6F000704A3431F9F7AEFD204604B070BD072012
:10C70000FBE770B5694DEB68052B01D0082070BDC3
:10C710006C682C2363436A4E641C64074436640FC0
:10C720009B196C60D98302211C46598408345C62D1
:10C7300000241C8401241C771A72120A5A72188071
:10C740005960FFF7D5FC002070BD57490089098C5E
:10C750000122D6E754490089098C0022D1E75249C9
:10C760000089898D0122CCE74F490089898D0022FB
:10C77000C7E74E494C4810B50023B8222031B838DD
:10C7800000F0F8FD00280CD0484A00219269FF23F0
:10C790002E244C43491C13550429F9D3052800D1F4
:10C7A000002010BD4049414810B50023B822B839D7
:10C7B000203000F055FD10BD10B53C48C068002881
:10C7C00004D03A48B821203000F024FE10BD37488C
:10C7D000C068052803D0072801D000207047012039
:10C7E000704710B50446008992DF010003D020464F
:10C7F000FFF79BFC10BD2D490320C86010BD00B59C
:10C800002A49B1B00522CA6000220A7001210091B4
:10C8100001686846884731B000BD8A7882700A880E
:10C8200002800A790271CA88C28009890181FF21C8
:10C830004181704770B5CA881346FF3B0B3B01D05E
:10C84000093301D1052102E0002A03D01146FFF788
:10C850006CFC70BD8A89144B002A19D0CA895E8A83
:10C86000551E1A4CAE4204D1098AA14210D19A82B7
:10C870000EE0DE8BAE4204D1098AA14208D11A84AF
:10C8800006E05E8DAE4203D1098AA14200D19A85AD
:10C89000198CFF2905D0998DFF2902D0FFF7AFFF32
:10C8A00070BDFFF777FC70BDBC330020AC220020C8
:10C8B00031F4000008C50100AF030000822302002C
:10C8C0006031002013C6010081C10100022900006F
:10C8D00010B50A88102A18D0112A19D0502A13D15D
:10C8E0000446881D097A01291CD002290CD101882F
:10C8F0002288914208D1017E1A30FEF7A6F900285D
:10C9000002D02046FEF702FA10BD8988418310BD8F
:10C910000021C943418300210177FEF78EF9FEF71C
:10C92000F9FC10BD0188A2899142FAD1C17E827EB4
:10C9300008021043C007C00F207710BD38B5044669
:10C9400008682061486860610020C0430D4660832C
:10C95000012168468170DF21C943018022461832D7
:10C9600069460120A0DF00280ED1FEF766F92046B7
:10C97000FEF7C2FC2946204600F028F8002803D123
:10C980002946204600F05CF838BD007F704710B59E
:10C99000438B4F4C86B0A34216D06B461A820022BE
:10C9A000009201920292039204891C8001249C70DF
:10C9B0009A8004AA03910292408B6946A6DF002860
:10C9C00002D0002006B010BD0120FBE770B58EB08C
:10C9D0000546012408A98C70DE20C04369460884FE
:10C9E0001C2101A804F0B5F969460879042108431F
:10C9F000694608714879002620434871701C000779
:10CA0000000F1030009648708878F9210840801C8B
:10CA1000E7210840204369468870142109A804F0E2
:10CA200098F969468C85CE851420088608A80A9155
:10CA30000990288B2B4609AA01A9A2DF0EB070BD70
:10CA4000F0B500250446681C01078FB0090F1031AE
:10CA5000684607950177681C0107090F1031684681
:10CA60004177817FF9273940891C81771C2104F0A7
:10CA700070F968460178102001436846017007A8E4
:10CA80000590012608A88671DD21C9436846818486
:10CA900008A808958178E7203940891C0140314376
:10CAA00008A8817014210AA804F053F909A80A9073
:10CAB00008A80B9068460686142145868186234681
:10CAC000208B08330AAA6946A2DF0FB0F0BD000030
:10CAD000FFFF000010B50A88102A08D0112A09D0DB
:10CAE000502A0CD0512A01D100F0A9F810BD898834
:10CAF000C18210BD0021C943C18200210AE0891D05
:10CB00000A8883889A42F4D1CA7E8B7E1102194327
:10CB1000C907C90F017210BDF0B500240546601C9D
:10CB200001078FB0090F103108A808940170601C2C
:10CB30000107090F103108A841708178F9263140AA
:10CB4000891C81701C2101A804F003F96846017951
:10CB500002200143F7200140102001436846017183
:10CB600008A801270690877156496846818439468E
:10CB700010310094017000200146684641708078B1
:10CB800008213040801C0843EF210840410849003B
:10CB90006846817014210AA804F0DBF809A80A90FD
:10CBA00068460B90078644860A218186A88A2B4610
:10CBB0000AAA01A9A2DF0FB0F0BD38B504460020D3
:10CBC000E060486820610020C0430D46E0820121FA
:10CBD000684681703B4922464631018014326946DD
:10CBE0000120A0DF002808D129462046FFF794FF46
:10CBF000002802D134480460002038BD007A704714
:10CC000010B5C38A314C86B0A34216D06B461A8247
:10CC10000022009201920292039204881C80012457
:10CC20009C709A8004AA03910292C08A6946A6DF8A
:10CC3000002802D0002006B010BD0120FBE770B52F
:10CC40008CB00546002000900190029001266A46B3
:10CC50000390167090800889298888422FD107A8F0
:10CC6000FDF77FFE0A21089804F000F804460A2127
:10CC7000099803F0FBFF072269460A74079A4A7471
:10CC800007990A0A69468A7407990A0C6946CA74A0
:10CC90000C75220A4A75220C8A75C875020A0A7632
:10CCA000000C48760A20488104A803908E71E88A17
:10CCB000A8DF002803D02969002900D088470CB0DC
:10CCC00070BD0000A1FE0000D4220020FFFF000084
:10CCD00014225043FE4A002180180171C1800222B3
:10CCE0000161C260416101817047FFB583B00F46A9
:10CCF000F84D069A05990646EB6811430320019109
:10CD0000002B01D0E96803E000290ED00121E96081
:10CD1000059A01249200240700920B0004F0ACF85D
:10CD2000073207213454748332000221EFE7EA48C6
:10CD30004169491C05D02169406989B203F096FF19
:10CD400000E060692169401E89B2484321690904F5
:10CD50008A0C216989B2794321DF002812D102218E
:10CD60000FE0384620DF00280CD10599002901D0BA
:10CD7000032106E0069900291FD13178042968D0E3
:10CD800020E0E96007B0F0BDD3484169491C05D0F7
:10CD90002169406989B203F069FF00E06069216997
:10CDA000401E89B241432069059A80B2784321DF51
:10CDB0000028E7D10699002901D00421E1E7317864
:10CDC00004292ED00521DCE7C3484169491C05D060
:10CDD0002169406989B203F049FF00E06069216977
:10CDE000401E89B248437188421800981018226981
:10CDF00092B27A4352180099531801461846069A7F
:10CE000021DF0028DBD0BDE72069718880B278433C
:10CE100080188A08316921DF0028B3D101990029DF
:10CE200017D00621ADE7AC484169491C05D02169FE
:10CE3000406989B203F01AFF00E060692169401E71
:10CE400089B24843216989B203F010FF20DF00282E
:10CE500098D1072195E7F8B59D4914230A780F204A
:10CE60005A435418241D9B4922788F88E668022A69
:10CE70001BD001252D07042A2AD0052A5BD1286959
:10CE800081B2304603F0F2FE0146A38828699A1960
:10CE900080B24843101A82086088181886192869D9
:10CEA0004B1C80B25843801B34E0B8026288216971
:10CEB000121A0918A3883018181801239B029A42E5
:10CEC00002D2920821DF31E0FF22013221DF2DE082
:10CED000A3687F481901CC3008180189428940684D
:10CEE000B04203D160885143814218D0032B16D041
:10CEF000286981B2304603F0B9FE0146286980B244
:10CF00004843301A820828694B1C80B25843638812
:10CF10009B19C01A83082046FFF7E7FE06E0286940
:10CF200081B2304603F0A2FEC01920DF002802D1F2
:10CF3000674901228A70F8BDF8B5654C069E657890
:10CF40000A2D1DD027787D19EDB20A2D01D30A3D97
:10CF5000EDB214277D432D1928716A6103C9296137
:10CF6000E860EB802E81A1780020002904D1FFF732
:10CF700072FF112800D100206178491C6170F8BD52
:10CF80000420F8BD38B50246514814230178504CAE
:10CF900059430818C368CC341B01E4580179C3888D
:10CFA000009343690C30A04738BDF8B5484B9978D9
:10CFB000012914D1002547499D70CA68082A05D067
:10CFC00002280FD003280AD10D2006E0022807D03E
:10CFD0000D7000F06FFA002801D0FFF7D3FFF8BD05
:10CFE000CD60F6E73A48142403783A4963431818A9
:10CFF0008B88001D5B1C9CB28C800378022B05D1B2
:10D000004688A102B14201D3012700E00027052B89
:10D0100001D1072A03D00021042B02D003E0012113
:10D02000FAE7072A03D00026042B02D007E00126E6
:10D03000FAE74088A302834201D3002A1AD00020D5
:10D04000314301433943C4D0224E2846F560FFF7EF
:10D0500099FF1F4C2078FFF73BFEB5806078401E9B
:10D0600060702078401CC0B220700A28B1D30A3802
:10D070002070AEE70120E3E7F8B50024154F14480F
:10D08000BC80FC6004704470847025462846FFF71D
:10D090001FFE6D1C0A2DF9D30F4D7C8068690F4E61
:10D0A000401C05D0306981B2686903F0DFFD00E003
:10D0B00070693169C01E89B24843B86004490020D4
:10D0C000BC80CC3102018C5052181481948107E04D
:10D0D000EC330020D82200200010001000000010C7
:10D0E000401C54810228EDD30820F8606869401C78
:10D0F00005D0306981B2686903F0B8FD00E070695D
:10D100003169401E89B24843316989B203F0AEFDEE
:10D1100020DF002803D1EE4A012191703970F8BD5B
:10D12000F8B50446EB480F46007800281DD0002CC7
:10D130001DD0002F1BD02068002818D001252D07F6
:10D14000A688286980B2864230D8102E2ED3E08877
:10D15000009000282AD0E0484169491C09D029697B
:10D16000406989B203F082FD04E00820F8BD0E207A
:10D17000F8BD68692969401E89B24843D54B0099BA
:10D180009D6871434B19984210D301200007006934
:10D1900080B2814208DD012000070069314680B27B
:10D1A00003F064FD002901D1B00701D00720F8BDCC
:10D1B000C8484288022A1BD0C5481101CC3024C778
:10D1C0000E18756023684350A0883081E088708114
:10D1D000A088E18800234843012109075B1C0C69F2
:10D1E0009BB2A4B2844205D20C69A4B2001B02E037
:10D1F0000420F8BD00200C69A4B265190C69A4B222
:10D200008442EBD9B348521C8560B3814280002030
:10D21000F8BD70B5AF4B1B78002B19D0002819D082
:10D22000002A17D00368022B10D2A94C1E01CC345F
:10D23000A559002D0AD04568301904896143691841
:10D240004589406865432818884205D8072070BD85
:10D25000082070BD0E2070BD13600020516070BDAD
:10D26000F8B504469B481E46007815460F46002830
:10D270001ED0002F1ED0002C1CD02068022815D2F2
:10D2800001019348CC304258002A0FD009184A892E
:10D2900008894968424351186268914206D9002DB5
:10D2A00004D0A84202D3A919814205D90720F8BDAC
:10D2B0000820F8BD0E20F8BD384600F0F5F800282B
:10D2C00011D0304600F0F0F800280CD0606800F073
:10D2D000EBF8002807D02B463A462146022000965C
:10D2E000FFF72AFEF8BD1020F8BDF8B504467948CE
:10D2F0001E46007815460F4600281ED0002F1ED06F
:10D30000002C1CD02068022815D201017048CC30B6
:10D310004258002A0FD009184A89088949684243AF
:10D3200051186268914206D9002D04D0A84202D358
:10D33000A919814205D90720F8BD0820F8BD0E20A3
:10D34000F8BD384600F0B0F8002811D0304600F0A3
:10D35000ABF800280CD0606800F0A6F8002807D0D1
:10D360002B463A46214605200096FFF7E5FDF8BD1D
:10D370001020F8BDFFB5574881B000781F4616460B
:10D380000C46002820D0002C20D0019800281DD069
:10D390002068022815D24E4D0001CC3529580029AD
:10D3A0000FD041194A890889496842435118626877
:10D3B000914206D9002E04D0B04202D3F119814225
:10D3C00006D9072005B0F0BD0820FBE70E20F9E7DD
:10D3D000019800F069F800281AD0384600F064F887
:10D3E000002815D0606800F05FF8002810D0606851
:10D3F0003246C119019803F093FC00962068002280
:10D4000000012D5803212046019BA8470020D9E7A1
:10D410001020D7E7F8B504462E480E4600780028BD
:10D4200024D0002C24D0206802281DD2284D0001D1
:10D43000CC352958002917D0401941890289406804
:10D4400051430918606881420ED900F02DF8002878
:10D4500010D021686068090149194A680989801A51
:10D4600003F004FC002907D00720F8BD0820F8BD10
:10D470000E20F8BD1020F8BD002002460090334673
:10D4800021460420FFF758FDF8BD1249097800290C
:10D4900006D0002806D00E49497801600020704768
:10D4A000082070470E207047800701D00020704789
:10D4B0000120704710B5064900204978002906D0A0
:10D4C000FFF7C9FC002802D0112800D1002010BDB0
:10D4D000EC330020D822002000100010FFB583B0EC
:10D4E000074600200C9C8646267805463AE0786878
:10D4F000A90041180A88684682804988C1800022B4
:10D50000694601A865DF002810D1684601780598B2
:10D51000814226D17046002801D0002200E002227C
:10D520002078891841181F2902D90C2007B0F0BDB6
:10D530007146002908D1401CC0B2411C069B049AC8
:10D5400021701A5401208646217806980A186946E7
:10D5500001A865DF0028E9D16946207809784018DC
:10D5600020706D1C3888A842C1DC7046002804D0A9
:10D5700020780699801B401E88550020D6E7F8B514
:10D580001546069C1E46074602220094FFF7A6FF9A
:10D59000002806D133461022294638460094FFF76A
:10D5A0009DFFF8BDF7B582B00026054616700068ED
:10D5B0001446002805D02846039900F0DFF806003D
:10D5C0002DD1687900281BD02078039F001D1F28CB
:10D5D00024D8684679DF002821D121780322481C0D
:10D5E00020707A5421781922481C20707A542078AF
:10D5F000C1196846008800F0BCF8217840182070F6
:10D600002989002923D001208446EA680398002A4A
:10D6100007D0227853189B1C1F2B04D90C2005B06F
:10D62000F0BD0720FBE71346521C491C2270C15471
:10D6300022786746511C2170875423782A8918184C
:10D64000E96803F06DFB2078297A4018207028697A
:10D65000002815D00021415622788C46D01C039911
:10D660001F28DBD8501C022320708B5422780A23F9
:10D67000501C20708B5420786246431C23700A543F
:10D68000A88A002809D028460094062202211430D6
:10D69000039BFFF774FF0600C1D1A88B002809D0B7
:10D6A00028460094072203211C30039BFFF767FFE5
:10D6B0000600B4D1A88C002809D028460094152271
:10D6C00014212430039BFFF75AFF0600A7D1E86A14
:10D6D000002805D02246039900F085F806009ED167
:10D6E000286B002805D02246039900F0BBF80600FD
:10D6F00095D13820405D002806D02246284603995F
:10D7000000F0E2F806008AD1304688E770B50D4691
:10D7100092B000216A46117007241171002812D0BE
:10D720000189002905D0C168002902D0097849077C
:10D7300002D4204612B070BD02A9FFF733FF0028C3
:10D74000F8D102AE00E00026002D0BD02889002879
:10D75000EFD101AA0AA92846FFF724FF0028E9D142
:10D760000AAA00E00022684603790178304672DF99
:10D77000E0E70870000A487002207047F8B5147896
:10D780000746A01C15460E461F2803D83879801C72
:10D790001F2801D90C20F8BD1D20001B80B269464E
:10D7A000864608803019801C7DDF0028F3D1386858
:10D7B000022805D168460088704501D8092107E094
:10D7C00038790821002801D0704501D968460088C1
:10D7D000421C3255641CE2B2B1542978801C0818EE
:10D7E00028700020F8BDF8B50D4611780646881D52
:10D7F00014461F2801D90C20F8BD33880720062BBA
:10D80000FAD31927FF01BB4202D94E4A9342F3D102
:10D810007288062AF0D3BA4202D94A4FBA42EBD1F3
:10D82000484FBB4203D0BA4201D09342E4D8481CCF
:10D83000052220706A5420781222411C21702A543B
:10D84000207841193088FFF794FF21784018C0B242
:10D85000207041197088FFF78CFF217840182070E4
:10D860000020F8BD70B5054600790E46801C1446B0
:10D87000C0B21178821C8A181F2A01D90C2070BDF1
:10D880000A46491C401C2170B0542078FF22411CDC
:10D8900021703254207881192888FFF76AFF217897
:10D8A0004018C0B22070AA88002A09D0A9680029AF
:10D8B00008D0801903F034FA2078297940182070B4
:10D8C000002070BD072070BDF7B582B002981446E5
:10D8D000406B0F46002832D002980025203000907F
:10D8E00028E00298416B0C2068430E1821783079AB
:10D8F0004A1CC01C2270785421781622481C2070C3
:10D900007A542078C1193088FFF733FF2178401806
:10D91000C0B22070B288002A09D0B16800290ED0A8
:10D92000C01903F0FDF920783179401820706D1C82
:10D930000098EDB2007EA842D3D800206FE6072001
:10D940006DE60000FFFF000030B5CB0008339DB24C
:10D9500093070024002B01D0072030BD564B9A605E
:10D960005219DA605C701C7058809980002030BDBC
:10D97000F7B5514C82B060880F4681426CD80020C8
:10D98000694608704E494D4E4868C005C00D16D016
:10D99000103807D50207120F083A92089200511862
:10D9A000C96904E08108474A890089180968800725
:10D9B000C00EC1400806850F012D01D10AE00425E3
:10D9C00068462EDF02280BD0002803D03EA2592142
:10D9D000F8F740FC6078A188884203D2401C02E03E
:10D9E00072B6F7E700202278C0B2904207D066787E
:10D9F0006078884201DA401C00E000206070012D50
:10DA00000BD062B6684600782FDF022805D00028C8
:10DA100003D02DA26121F8F71DFC2848864219D0B9
:10DA2000A068F50004994151029900290CD0002FFB
:10DA30000AD060883A464643E068301803F070F92F
:10DA4000A0682818878002E0002128188180002023
:10DA500005B0F0BD0420FBE70920F9E70EB504E0AE
:10DA600068468188029A0098904702AA01A96846F0
:10DA700000F003F80028F3D00EBD70B50E4B05245E
:10DA80005D781E78B54215D01D781C789E88B4420A
:10DA900001DA641C00E000241C705C88DE686C43C2
:10DAA000A41904609B68E800C418A4880C80185866
:10DAB00000241060204670BDE8220020FFFF000017
:10DAC00000ED00E000E400E02E2E5C2E2E5C2E2EF9
:10DAD0005C2E2E5C2E2E5C536F757263655C6170DC
:10DAE000705F636F6D6D6F6E5C6170705F736368A4
:10DAF0006564756C65722E63000000008307FF2269
:10DB0000DB0E9A408907090E994000280BDA0007BE
:10DB1000000F08388308FF489B001B18D869904302
:10DB20000843D86170478308FB489B001B1818689E
:10DB3000904308431860704770B50124F7496004AA
:10DB40000860F74940108860F54940398860F54D14
:10DB50006C602F20F8F7EEFAAC60F34D00242F2014
:10DB60006C61F8F7E7FA2C7170BDF0B5EE4F282123
:10DB7000BC6841430D1939694A1C09D028224A431F
:10DB80001619AB68B268934204D8D21AB2606962BF
:10DB90003861F0BD0A4602E00A46796A9B1B4E1CBA
:10DBA0000BD028264E433719BE689E42F4D3282650
:10DBB0004E433619B768FF1AB760AB606962282117
:10DBC0004A4311194862F0BDF8B5D74C2569681C65
:10DBD00036D0D648002640686169401A07023F0ADD
:10DBE0001AE028204543A0682A189068B84215D842
:10DBF000A3693F1A8619556A002B0AD0116AD069A9
:10DC00009847002808D0FF21C9A26431F8F722FB09
:10DC100002E0D169106A8847681CE2D1A178E078F7
:10DC2000814206D1401CC0B2E070022801D1002020
:10DC3000E070BD490006800D1C310E5000F0F4F973
:10DC4000F8BDF8B50446B84801690091467856E039
:10DC5000B548F100C2688D184BE0601C07D0B24A8D
:10DC6000282192686143204689184C6A20E0287870
:10DC7000182141436A68401CC0B252182870A97824
:10DC8000884201D100202870A74B506828219B684A
:10DC90004143C9181368012B2DD10B7E002B2AD1CB
:10DCA0009368CB60D3680B6113694B6152690A6258
:10DCB0009D4ACF685369BC46FA1A1202A84F120A4D
:10DCC000BA4202D20B69D21809E062469A1A1202CD
:10DCD0000B69120A934201D99A1A00E000228A6065
:10DCE0000022CA600A6101220A76921E4A62FFF788
:10DCF0003CFF601CB1D1287869788842ADD13046AC
:10DD0000761EF6B20028A3D18748016900988142A7
:10DD100001D00120F8BD0020F8BD92490020086024
:10DD200048608860C8608F494039086048604BE7A8
:10DD3000F0B5002087B0C04302907B484669056972
:10DD4000684600F076F9074600F090F90446002F87
:10DD500008D002AA3146009800F0D0F90298FFF7E7
:10DD600070FF06E00298FFF76CFF002801D1002C3D
:10DD700002D0284600F0EBF907B0F0BDFFB59807D8
:10DD8000002481B01E4615460F4600280BD1002EF8
:10DD900009D0FFF7D1FE64490A9888610F703246B6
:10DDA00000208E6008E0072005B0F0BD2823434323
:10DDB000D4509B181C76401CB842F7DB2820474300
:10DDC000BB19032048700F461846CB60194618301F
:10DDD000002218232E465E43D3005B181C705C7033
:10DDE0009D7058603018521C032AF5DB0020C04398
:10DDF0003861BC70FC7001245B4824050460032179
:10DE00001420FFF77BFE454880380460474C01989A
:10DE1000A06003211120FFF771FE60687861002087
:10DE2000C2E770B5404CA568002D06D0002A06D088
:10DE3000002804D00023247809E0082070BD0720C2
:10DE400070BD28265E43AE59002E04D05B1CA34251
:10DE5000F7DB042070BD282401265C432E51641991
:10DE6000E26161600360002070BD2A494868C00516
:10DE7000C00D17D0103807D50207120F083A9208C4
:10DE800092005118C96904E08108234A8900891861
:10DE900009688007C00EC1400806800F012803D022
:10DEA000032803D0022070470020704701207047EC
:10DEB000FEB504461C48174682680D46002A0CD061
:10DEC00001788C4201D2052D01D20720FEBD2146EA
:10DED000282359435358012B01D00820FEBD881830
:10DEE000406801284AD00026FFF7BFFFC0000E4956
:10DEF0000190C9684018694600F06FF900283FD0CA
:10DF0000012144600160094949680830E2C00649BE
:10DF100001982BE000ED00E000E400E080E100E08B
:10DF20004013014000100140F8220020001501407C
:10DF30002E2E5C2E2E5C2E2E5C2E2E5C2E2E5C53F6
:10DF40006F757263655C6170705F636F6D6D6F6E2E
:10DF50005C6170705F74696D65722E630000000013
:10DF6000FFFF7F004011014080E200E0C9684118D6
:10DF70000098487000F058F80020FEBD2E46B3E728
:10DF80000420FEBDF8B5B64D0446A868002809D0A7
:10DF900029788C4201D30720F8BD282161434058DD
:10DFA000012801D00820F8BDFFF75FFFC600E86830
:10DFB0006946301800F011F9002809D0022112C07A
:10DFC000E86831180098487000F02EF80020F8BD7D
:10DFD0000420F8BD38B5A24CA068002815D0FFF782
:10DFE00044FFC500E0686946281800F0F6F80028EC
:10DFF0000DD003210160091F4160E06829180098D5
:10E00000487000F011F8002038BD082038BD042009
:10E0100038BD94494968016000207047401A0002E9
:10E02000000A10600020704701208F490005086039
:10E03000704710B58A4900238A78CC78A24212D062
:10E04000521CD2B28A70022A00D18B708A78844B1B
:10E0500092001C339A580260486910180002000AA6
:10E060004861012010BD0360002010BDF8B57C4858
:10E0700001690091457833E07948E900C0680E18DD
:10E0800034782AE0182060437168641C0818B1785D
:10E09000E4B2A14200D100240168022902D0032980
:10E0A0001BD113E06E4A40682821926841438F18C3
:10E0B000397E002911D000F0A2F8002038760CE05B
:10E0C00028277843C0180276406A03E0644900229A
:10E0D0008B680869471CF3D108617078A042D1D1E0
:10E0E00028466D1EEDB20028C6D15D480169009832
:10E0F000814201D00120F8BD0020F8BDF7B5584C91
:10E100000025A76823691EE028215943C9198E6894
:10E11000864202D9301A886017E0801B75190026E4
:10E120008E600E764E699C464B6AB646002E0AD02B
:10E13000019E76193602360ACE6076460E61166862
:10E140004E6261461160591CDED12361FEBDF8B5F7
:10E15000434801694A1C3DD02822514382688918EE
:10E160008E6840494C6847690079E11B0D022D0A11
:10E17000ED1C002815D101203C4A000450603B4AA8
:10E18000403A5060384940008031086038490860A2
:10E190003849012008602F20F7F7CCFF30490120D3
:10E1A0000871B54200D23546E81900022D49000A2F
:10E1B000403108602B494968001B091B0902090A04
:10E1C0000002C91C000A814203D9012026494004EB
:10E1D0000860F8BDFFF7B0FCF8BD42788378521CA8
:10E1E000934200D100220378934201D1002070476E
:10E1F0000A6041684078182250430818704770B58B
:10E20000174E3569B26829460C4606E0844207D0AD
:10E21000254628235C43A3185C6A631CF6D170BDB5
:10E22000002BFCD0A54208D1282041438818406A21
:10E230003061401C01D1FFF77FFCB16828204443C6
:10E240006018282382685D43406A6B185862431C3B
:10E25000E5D028235843401881688918816070BD33
:10E26000F82200200015014000E200E040130140C8
:10E2700000E100E00010014038B57A497A4A488848
:10E2800090420FD04A78794C521CD2B24A70237B0C
:10E29000934208D3083175DF002803D0A169002913
:10E2A00000D0884738BD00254D70217C002907D05B
:10E2B0003B2176DF002803D0A169002900D08847E0
:10E2C00061690029EED068460095884738BD70B571
:10E2D000054601461C22654802F022FD614C0026DD
:10E2E00026702968002907D00822A01802F018FD1E
:10E2F000204608307ADF02E05A4808307BDF0028E9
:10E3000008D1401E608057486670594A0021001DA0
:10E31000FFF787FD70BD10B552484068FFF732FE29
:10E3200010BDF8B54F48103000F08EF800264D4D66
:10E330004E4C002806D06169002919D001200090B8
:10E34000684614E02878002804D0616900290FD0BD
:10E350000096F5E7687800280CD0A168002268686C
:10E36000FFF7A6FD002803D0A169002900D0884747
:10E370002E70F8BD6168F1E7F8B53C4C02880027C3
:10E38000384DE689102A18D029464968112A21D02B
:10E39000122A2DD0502A0FD1801D0288B2420BD1F3
:10E3A000028B022A08D1C27E837E10021843C00766
:10E3B000C00F13D0FFF7B5FFF8BD81886980014613
:10E3C000284808220E31103002F0AAFC6F70002E8F
:10E3D000F0D0F8BD0020C04368806F700846FFF79A
:10E3E000D1FD0028F5D0A1690029F2D08847F8BDF9
:10E3F000811D1C480822103002F092FCDAE7F8B5C3
:10E40000014618480822083002F08AFC15480830F6
:10E410007ADF04000DD11348103000F015F8012503
:10E42000002808D011484169002902D068460095AB
:10E4300088472046F8BD0B4E35703146083170884C
:10E4400075DF04467570F4E7418806480830028895
:10E45000914204D34088814201D8012070470020B6
:10E46000704700001C230020FFFF0000D83400206C
:10E4700079E2010010B508461146F7F7F3FE10BD2A
:10E48000F8B53D4C2078002837D02069002807D007
:10E490000026E068002805D00025002E04D013E0F7
:10E4A0000126F6E70125F8E7684651DF052806D082
:10E4B000002806D031A26921F7F7CCFE04E001263E
:10E4C00002E0216900988847002D12D160886946D2
:10E4D0000880A06861DF052806D0002806D027A2A2
:10E4E0008021F7F7B7FE04E0012502E0E168A068AB
:10E4F0008847002ED8D0002DCFD0F8BD70B50029A8
:10E5000001D08C0701D0072070BD1B4C0125A160F4
:10E5100062802849636010DF0028F5D1257016203D
:10E5200026DF70BD11DF002801D0012100E00021AD
:10E53000114A11707047002803D00F49C8600020AD
:10E5400070470E207047002803D00B490861002057
:10E5500070470E20704710B507484068002808D063
:10E560008047002804D0FF2104A23331F7F772FE60
:10E5700010BDFFF785FF10BD342300202E2E5C2E2A
:10E580002E5C2E2E5C2E2E5C2E2E5C536F757263CD
:10E59000655C73645F636F6D6D6F6E5C736F6674E3
:10E5A0006465766963655F68616E646C65722E632D
:10E5B0000000000075E4010010B56C4AD368002B20
:10E5C0000AD0CAB2017880689847002803D068A2B0
:10E5D0002821F7F73FFE10BD012906D00029FAD106
:10E5E000037882681846904710BD0378012182683D
:10E5F000F8E7F8B55D4D6946687801F050FB0028F2
:10E600001ED12F4600241437012616E00C2069681D
:10E6100060434018037831463A6899400A4210D066
:10E620008268002A0DD04178012901D1002100E043
:10E630000121FFF7C1FF641CE4B228788442E5D3CE
:10E64000F8BD7A680A42F6D081680029F3D0417893
:10E650000129EDD0EAE770B5444D04460E4628691D
:10E66000FFF790FC002809D128461430066044606A
:10E6700034432246A9682869FFF71AFC70BDF8B533
:10E68000052A01D20720F8BD384C454D6060217045
:10E69000E360A260002201240CE00C234B431B1812
:10E6A0001E785F68B600BF00761937601E78234673
:10E6B000B3401A430B46491EC9B2002BEDD12B487B
:10E6C000384B1146401C01F06AFA0028DBD127487C
:10E6D000354A00211030FFF7A4FBF8BD10B52348E0
:10E6E0004168002903D0407801F07CFA10BD082071
:10E6F00010BD10B51D4C6068002808D0607801F08E
:10E70000B2FA002802D12069FFF73CFC10BD0820B6
:10E7100010BD38B5154A0C461178884201D907203A
:10E7200038BD0C2148435168451800290CD0694672
:10E73000507801F0B4FA0028F2D16A780121002A59
:10E7400004D0012A08D00FE0082038BD2B78009AA9
:10E75000DA40D20707D104E02B78009ADA40D207DA
:10E7600001D0217000E02070002038BD4823002037
:10E770002E2E5C2E2E5C2E2E5C2E2E5C2E2E5C53AE
:10E780006F757263655C6170705F636F6D6D6F6EE6
:10E790005C6170705F627574746F6E2E6300000050
:10E7A0000007005057E60100F3E5010070B5FD4B8E
:10E7B00004469E7A082000250E4207D0FA4884427B
:10E7C00002D01889A04202D10020156070BD05203A
:10E7D00070BD70B50546F3491C206843A039441844
:10E7E00020461130062102F0B4FA2046102102F032
:10E7F000B0FAFF2121740020A176C043208328466F
:10E8000000F050FE70BDF7B5E64F05250024064622
:10E81000A03F002E0AD01C206043C01910300722F0
:10E82000314602F0A8FA002807D00AE01C20604315
:10E83000C019018B0298814203D101980025046020
:10E8400002E0641C042CE4D32846FEBD0C2148439E
:10E85000D44910B5012240188272911E0181FF2116
:10E86000C172072102F075FA10BD00207047F0B5A3
:10E8700087B00D46074614206946888268780C21C7
:10E880004843C84E05AA801900896946AADF0028B6
:10E8900033D1687818214843741A00196946001D5D
:10E8A0008A8A02F068FA0028687806D0182148435E
:10E8B000215800290DD0BD4E0CE00C21414389198F
:10E8C000897A890719D418214843001902F041FABE
:10E8D00013E0B74E69468A8A225068781821484367
:10E8E0000019001D694602F01BFA68781821484398
:10E8F0000119342318223846B047002007B0F0BD74
:10E9000070B50D4601466878A64C18225043183C55
:10E9100000193423FEF72EFD002806D1697818224D
:10E9200051436258521C00D1625070BDF8B5407816
:10E9300018239C4C4343183C9A4E0C270021E55861
:10E94000784380190A46002D07D0867A770604D5C9
:10E95000B60602D41919091DAAB20089A9DF002838
:10E9600000D09448F8BD002806D0FF210170417006
:10E970008170C170002070478E4833387047FFB5F2
:10E9800088488BB00C300068149F1E4600286AD05F
:10E99000502F68D803A8FFF7E6FF002803D0864A67
:10E9A0008649F7F757FC00256846057305702C4625
:10E9B00004970596A1B208AA8148FEF72AFC002810
:10E9C00006D1082208A90B9802F0D5F9002818D022
:10E9D000641C042CEED36846847BFF2C43D00C9837
:10E9E000042811D06F481C21A038301A02F03EF9DB
:10E9F0000127042824D204A801900D98002811D0E2
:10EA000017E068468473E6E7502F09D04020694636
:10EA1000087068460178032001436846017047E0AA
:10EA20002020F4E738466649A0400C39496808427E
:10EA300019D0204600F036FD2020694608702EE0EF
:10EA4000584818213038301A02F010F900280CD03C
:10EA5000544C1821183C301B02F008F9002811D042
:10EA60004020694608700FB0F0BD04A80190202036
:10EA7000694608701C2044434A484D73A03820184A
:10EA800005900CE03021684601704573C773454816
:10EA9000807A800703D42046182102F05AF90C9896
:10EAA0006946032808780BD002210843694608709C
:10EAB00004A80190694603A80D9A00F035FDD2E73D
:10EAC0003843F4E7F0B585B0040035D0354900256A
:10EAD0000C310D6028468D72FFF7B8FE31481821C1
:10EAE000183802F036F90026FF273046FFF771FE8E
:10EAF0003348001F8755761C042EF6D350216846F4
:10EB000081800421C1802F4800902D496846FEF77E
:10EB100007FB00280ED12A4E01200C3E30702078D1
:10EB200000280CD069468888C988484381B22448A7
:10EB3000FEF770FC05B0F0BD1E483338FAE7194FF8
:10EB40000024A03FA1B202AA1D48FEF762FB0028E4
:10EB500009D11C206043C01900231C2202A9FEF722
:10EB600009FC002801D03570E4E7641C042CE9D3CB
:10EB7000E0E770B5064612480D460C3800780028CC
:10EB800022D00C493339002E20D0002D1ED0286809
:10EB900000281BD0034C0C342168002918D00548EC
:10EBA0003D3870BD94350020FFFF0000EBD201001E
:10EBB00061D2010041800000F4230200C304000080
:10EBC000702300207FE90100FE48EAE70846E8E7F5
:10EBD00020600622A91D201D02F0A2F82879A0724B
:10EBE00000203070DDE710B5F749F64B09780029B1
:10EBF00010D0002803D0017800290BD102E0F148A1
:10EC0000801D10BDF1490A68002A03D04078002811
:10EC10000ED101E0184610BDEC4A0C3A947A012C52
:10EC200006D01846A307F6D51089091D7EDF10BD52
:10EC3000E448083010BD10B5E34AE24B1278002AD0
:10EC400013D09A1D002805D0002903D00278002A8D
:10EC50000BD101E0104610BDDC4C00222468002CD2
:10EC600003D0407800280BD101E0184610BDD748EA
:10EC70000C38807A012803D0430704D5012005E031
:10EC8000D048083010BD400602D50220086000E0E0
:10EC90000A60002010BDF0B5CB4A1378C94A002B9A
:10ECA0001AD0931D00280BD0002909D00C68002C25
:10ECB00006D08C68002C03D0007800280CD101E02D
:10ECC0001846F0BDC1480068002805D00023BF4D9C
:10ECD00018461A46AC3D19E01046F0BD1C245443BA
:10ECE0006419A67EF60706D18E688700F451B64EE9
:10ECF00008363254401CA67EB60704D410349F0058
:10ED00000E685B1CF451521C042A05D20C799C42FB
:10ED100002D90C7B8442E1D80B7108730020F0BD4E
:10ED2000A8488830704710B5A7490A78A549002A35
:10ED30001AD0002803D00278002A15D102E0A14899
:10ED4000801D10BDA14A1268002A0DD080780428C9
:10ED50000CD29E4A1C214143AC3A8918897EFF2976
:10ED600004D000F0CCFB10BD084610BD954808301B
:10ED700010BD70B594490A789249002A1DD0002828
:10ED800003D00078002818D102E08E48801D08E7E3
:10ED90008E480068002810D000208C4D0446AC3D01
:10EDA0001C2161434919897EFF2902D0204600F0C9
:10EDB000A6FB641C042CF3D3F3E60846F1E67CB50D
:10EDC000044681480D4601787E4800292DD0811DDA
:10EDD000002C29D0002D27D02178002925D17B496E
:10EDE0000968002921D077496078083100281BD1B3
:10EDF00076480C38807A012816D0A078042813D2DF
:10EE00001C225043714AAC3A8018807EFF280BD0F8
:10EE1000A96800290ED06A68002A0BD0142A09D2EA
:10EE20002878012802D005E008467CBD67482038D4
:10EE300001F076FF6448A1786A460C30FEF7E9F9E4
:10EE40002878634980000A582146684690477CBD6F
:10EE50007CB505465C480C4601785A48002921D00B
:10EE6000811D002D1FD0002C1DD02978002919D11B
:10EE700056490968002915D0A878042815D21C2104
:10EE800048435249AC394018807EFF280DD068783D
:10EE90004E4A0C2141430C3A8918897A890707D4D4
:10EEA000484889307CBD08467CBD464808307CBD5A
:10EEB000A168002911D1616814290ED22178012995
:10EEC0000BD1182148434149182224394018001D0C
:10EED000A06068785043085860603B48A9786A464B
:10EEE0000C30FEF796F920783949800010310A5825
:10EEF0002946684690477CBD33490A783149002A43
:10EF00001AD0002803D00278002A15D102E02D483B
:10EF1000801D70472D4A1268002A0DD08078042881
:10EF20000CD21C2148432949AC394018807EFF2867
:10EF300004D024488830704708467047214808307C
:10EF400070472048893070471E48893070471D48F7
:10EF5000893070471C4A13781A4A002B11D0931D30
:10EF6000002905D0002803D00078002809D101E04D
:10EF700018467047154B1B68002B02D00870002004
:10EF8000704710467047FEB50E46044681780E481D
:10EF90006A460C30FEF73DF9002832D160780B4FFD
:10EFA0000C2148430C3FC019807A80062AD4022ED7
:10EFB00028D0012E28D0074DA0781C2148430349B2
:10EFC000AC3909E00880000064230020A03500204F
:10EFD000C42302006BE80100411800231C2268468C
:10EFE000A847002812D0022E0BD020780C214843CD
:10EFF000FA494018807AFA4980000A582146684642
:10F000009047FEBDF74DD7E7F74DD5E7022EF8D074
:10F0100060780C214843C019817ADF221140817247
:10F02000607818214843ED491C233C3941181822C7
:10F030006846A847D9E770B5EC4D04462A78EC48F5
:10F04000002A1BD0821D002C17D0002915D0227851
:10F05000002A13D1E14A1268002A0FD0A0780428B0
:10F060000DD21C225043DD4AAC3A8018827EFF2A22
:10F0700005D06278FF2A05D017E0104691E5DC48FC
:10F0800008308EE50A78022A0FD01030072201F0EE
:10F0900047FEA17801208840696808436860022122
:10F0A0002046FFF770FF00207BE5D148401E78E541
:10F0B0000B4610B5CD49CE4A097800292DD0911DB7
:10F0C000002805D0002B03D00178002925D101E0CC
:10F0D000084610BDC149096800291ED0C44A81787C
:10F0E000D21EFF2909D01C204143BC48AC38091866
:10F0F000887E800711D410310AE04078FF280CD0B8
:10F100000C214843B5490C394118887A800704D549
:10F110000722184601F004FE0022104610BD1CB55F
:10F1200004468178B1486A460C30FEF772F8002830
:10F1300013D1607818214843A8491C233C39401852
:10F1400018226946FEF716F9A448A549807A80007E
:10F1500010310A582146684690471CBDF0B5054657
:10F1600087B0FF24A1480594007800286ED09B4FFB
:10F17000386800286AD001A8FFF7F5FB002804D002
:10F18000974A9C493032F7F765F80020064606900A
:10F19000281D0390342069460882FF2088710020D2
:10F1A000087100908D4C28880C3C10280ED00A461F
:10F1B000A8880221FFF7FAFA002807D100980C214D
:10F1C00041430919CA7A69468A7148712988142904
:10F1D00078D02EDC10293BD0112975D0132935D1D8
:10F1E0001320694608723A1DA88800217FDF002895
:10F1F0002CD100980C21414309198A7A04231A431F
:10F200008A72C97AFF2913D016216A461172182111
:10F210004843724924394018001D142101F099FD1A
:10F2200000980C2148430019817A202211438172F1
:10F2300024E117297ED06A48203018297BD0522932
:10F2400004D1B97A8900415801A8884707B0F0BDB8
:10F25000694F6A4601213846FFF7A8FA0028F5D120
:10F2600000990C20484302220019827211236A4639
:10F2700013725171A98801810722A91D01F050FD67
:10F28000687BC10707D0410858480830405CFF2818
:10F2900008D0059006E03A4605A9A81DFFF7B3FA85
:10F2A0000028C5D100990C22514309190598C8724C
:10F2B0008A7A08231A438A726946887101A8FFF77F
:10F2C0002EFFDBE024E0FFE700980C214843011902
:10F2D000887AFD2210408872010706D540060DD5B8
:10F2E000002101A8FFF74FFE08E068468079FF285B
:10F2F00004D0FFF76EFAFF206946887100980C224F
:10F300005043102100198172122069460872B5E03D
:10F3100000980C2148430019C07AFF281FD1EA89C0
:10F3200005A90020FFF76FFA002811D100990C22DF
:10F33000514301E020E08EE009190598C8728A7AED
:10F3400008231A438A726946887101A8FFF7E7FE0D
:10F3500000980C2148430019C07AFF2807D0009874
:10F36000182148431D493C394018001D0690A888C3
:10F370000022069981DF69E700980C2141430919B1
:10F380008A7AFB231A408A7214216A461172A9797B
:10F39000002901D00E4671E0182148430F4914227C
:10F3A0003C394018E97A8170A97A41702946001DDC
:10F3B0000C3101F0B5FC00980C2148430119887A02
:10F3C00042065BD5082210438872CA7AFF2A15D0FC
:10F3D000202210438872002139E00000A03500206F
:10F3E000C4230200EBD2010061D20100642300209B
:10F3F0000880000037090000FFFF000005A800F0AA
:10F4000058F8002801D0064638E06946059888710A
:10F4100000990C224A431219D0721C23504F5843B2
:10F42000AA89C0190283E87A40070FD51C204143FE
:10F43000C81929461022203101F072FC00981C21C5
:10F440004843C019817E490849008176012101A8FD
:10F45000FFF799FD12E000990C22514309198A7AAD
:10F4600040231A438A7215216A461172B97A8900BB
:10F47000415801A88847002800D03A4E02A93246D8
:10F4800001A800F051F86846007A122800D0DDE6A5
:10F4900000980C2141430919897A0129F7D0FFF717
:10F4A000D5F9D3E6012181402F4842688A43426062
:10F4B000704770B52B4A0546921C294800241C232E
:10F4C00063431B189B7EFF2B04D0641C042CF6D3D3
:10F4D00010465CE40A78022A09D01C226243101804
:10F4E000FD2282761030072201F01AFC04E01C2174
:10F4F00061430818FE2181762C700022E8E77CB574
:10F50000054681B218486A460C30FDF782FE0400B9
:10F5100008D150216846FDF77DFF040002D128463E
:10F52000FFF757F920467CBD0D4BAC331B681847DD
:10F53000002070470020704710B5FFF798F910BD04
:10F54000002070470020704710B5FFF7D9F910BDB3
:10F55000002070470020704710B5FFF7E7F910BD95
:10F56000F434002041800000642300207CB515465F
:10F570000E46040003D1EFA2AF21F6F76BFE206A1E
:10F58000002809D0F74840680190009668468580B9
:10F59000226A0199009890477CBD70B50C46050021
:10F5A00003D1E4A2A121F6F755FE002C04D1E1A27B
:10F5B000A2210020F6F74EFE00202860208070BDBA
:10F5C00010B5E948816801290AD1E8494968490725
:10F5D00006D500218160084600F0F2F900F073F9C9
:10F5E00010BD7FB514000D46064604D1D1A271218D
:10F5F0000020F6F72FFE266065600020A060A08145
:10F60000E0812061A082E0826083208320772062F5
:10F610006062203420726846007B60727FBDFFB557
:10F6200081B00A9F1C461500064604D1C1A2922152
:10F630000020F6F70FFE002C04D1BEA2932100207B
:10F64000F6F708FE002F04D1BAA294210020F6F7A5
:10F6500001FE2E60002E01D0029800E000202080E4
:10F660000020388005B0F0BDF8B50C00064604D087
:10F6700000F0A6F9050008D101E00E20F8BDFF2139
:10F68000ACA213310020F6F7E5FD002E0AD1E07E92
:10F69000002801D0012300E000232A460321B448BA
:10F6A000FFF79FFF217C01200246B24E8A40B260E4
:10F6B000216903228B00B0495B181A60237C9840B3
:10F6C000B0606068800040180260E0688000401808
:10F6D0000260A0680027800040180760207C28771F
:10F6E00060682968361589198860E0682968891971
:10F6F000C860A06829688919086120682968891983
:10F700004862A07E617E400089000843217E084354
:10F71000296815229201891848612868FF30013054
:10F72000876068682ADF002804D0FF2181A2423167
:10F73000F6F790FD217D68682BDF002804D0FF21BB
:10F740007CA24331F6F786FD2F622968042003224C
:10F75000120289184860686826DF002804D0FF215B
:10F7600074A24A31F6F776FD2968012089190860EC
:10F77000022068620020F8BD10B500F021F90400F5
:10F7800004D1FF216BA25E31F6F764FD60682ADFC9
:10F79000002804D0FF2167A26131F6F75BFD6068A5
:10F7A00027DF002804D0FF2162A26231F6F752FD64
:10F7B000226800210520000212181160217F012219
:10F7C0008A406C49CA60FF21217700212268C94321
:10F7D0001218916022681218D16022681018016115
:10F7E0000023224619461846FFF7FBFE10BDFFB561
:10F7F00083B0174600F0E4F8040004D1FF214DA2C5
:10F800009A31F6F727FD0026694625460E71203508
:10F81000687A002807D001A82EDF00280CD0FF212D
:10F8200044A2A53106E0606827DF002804D0FF214C
:10F8300040A2AA31F6F70EFD606A02280CD011260C
:10F84000687A002833D0684600792FDF002837D047
:10F85000FF2138A2D63131E00C98B84201D90146D7
:10F8600000E03946002920D001206062002060833A
:10F870002872218320460E30831E821F0090394655
:10F880000498FFF7CCFE20461630831E821F00909E
:10F890000C990698FFF7C3FE207F0121814035486F
:10F8A000C160204600F092F8CAE70726C8E7606802
:10F8B00026DF002804D0FF211EA2DB31F6F7CAFCA8
:10F8C000304607B0F0BD70B5040003D119A2D821AD
:10F8D000F6F7C0FC608B401C608320462030017A24
:10F8E0000125002904D10572628B2046FFF73EFEF8
:10F8F00020680522120280188069C1B220690028A0
:10F9000009D0E08AA38A984205D2E08A23691B18AD
:10F91000401CE0821970E089218B884235D2A068B2
:10F9200000282BD0E089A189884227D2A068E189EC
:10F93000405C24E02E2E5C2E2E5C2E2E5C2E2E5C47
:10F940002E2E5C536F757263655C7370695F6D61B9
:10F95000737465725C7370695F6D61737465722E28
:10F96000630000003C2402000031004000330040EE
:10F9700000300040000500500007005000202168C2
:10F980008918C861E089401CE081608B218B884226
:10F9900015D3207F854026488560E58921460C31B6
:10F9A000081FFFF7FAFD21461431081FFFF7F5FD88
:10F9B000022060622A4601212046FFF7D7FD70BD74
:10F9C000002801D0002070471A48704710B5040085
:10F9D00003D1194AC021F6F73DFCA068002807D0E2
:10F9E000E089A189884203D2A068E189405C00E0F7
:10F9F00000202268052109025218D061E089401CCC
:10FA0000E081E089228B904211D2A068002807D0C3
:10FA1000E089A289904203D2A068E289805C00E07C
:10FA2000002022685118C861E089401CE08110BDA7
:10FA300000050050AC35002034F9010031B5054C0B
:10FA400004E0401E00902046F6F784FB0098002852
:10FA5000F7D138BDE7030000F0B5002201230326EB
:10FA600036041F4697400C463C420FD0C5682C46D2
:10FA70003C420FD03446BD43C560934D97007D197D
:10FA80002F68B7432F602F6827432F60521C202A0E
:10FA9000E7D3F0BD012464043D43EDE7F8B58B489E
:10FAA00005698B490020C863074632E014213A46B5
:10FAB0004A434168806854180121B940014226D068
:10FAC000E068C64320686E40064031462046FFF796
:10FAD000C3FF7E48006968400CD00543E068216898
:10FAE000C04368400840014600902046FFF7B4FF3D
:10FAF000009806433046A168A84301402A46606842
:10FB00003240104002460A4301D0226990477F1CD0
:10FB1000FFB2704841788F42C8D3F8BDF0B56D4A46
:10FB200000215368142250430124674D03273F04EA
:10FB30001E5822468A40164206D08A00521916687C
:10FB4000BE43166016681660491C2029F0D3F0BD2C
:10FB500010B5002903D08A070024002A01D007200D
:10FB600010BD5C4A0B465160107014215470414323
:10FB70001846946001F0EDF800205749C0438860B2
:10FB8000564840210160564A1068FF231B049843E1
:10FB90000B041843106053480160002010BDF8B5F5
:10FBA0004C4F84467D68002D07D0002B07D0787815
:10FBB0003C78A04205D30420F8BD0820F8BD0720FA
:10FBC000F8BD0E461424164344432E516419236194
:10FBD000A260616061460870411C7970FFF79EFF6A
:10FBE0000020F8BDF0B53B4A5168002904D0537895
:10FBF000984203D30720F0BD0820F0BD344B002508
:10FC0000DD63324B1C699768002F02D1324EDB0551
:10FC10007360012686403E4396601422504342188A
:10FC2000D560002201230D5893401D4216D0254671
:10FC30001D4202D003252D0405E001256D04461860
:10FC4000F7681F43F760204B9600F3181E680327E0
:10FC50003F04BE431E601E682E431E60521C202AB5
:10FC6000E0D30020F0BD70B51A4C0546606800284E
:10FC700004D06078854203D3072070BD082070BD92
:10FC80002846FFF74BFF0121A068A9408843A060E8
:10FC900003D101201049C0078860002070BD0D4BC2
:10FCA0005A68002A04D05B78984203D30720704733
:10FCB00008207047142358438018044A12690068CA
:10FCC000024000200A607047000700500005005005
:10FCD00040610040782300200063004080E200E0A3
:10FCE00004E400E000E100E010B5FF210D31FE4822
:10FCF00001F02FF8FC48E621E83801F02AF8FA482C
:10FD00000F2140308172F8490E20E839C881FF2167
:10FD1000F548D731018100214160012010BD70B547
:10FD2000F14CA034227B002A32D0EF4AE83A127814
:10FD3000092A25D00122ED4B984202DA258AAD1816
:10FD4000258219256D01A84202DD608A8018608233
:10FD5000994202DAA08A8018A082A94202DDE08AD4
:10FD60008018E08200200E21DF4A615E43009B186C
:10FD7000B0255D5F8D420CDD217E012902D005E0BA
:10FD80000522D8E7D8498031C96B88470020207305
:10FD900070BD401C00B20428E8DB70BDF7B5192324
:10FDA00000985B01C218D04C029825460027FF300E
:10FDB00059002C308035A0343E468A4202D9CC4AC4
:10FDC000904206D9019AD2188A4212D9C84988426B
:10FDD0000FD8C5480127E838C088A0802680A079C0
:10FDE000012806D1A671E079012802D1A96A002074
:10FDF00088470199AF22FF3100205F319200914284
:10FE00000AD8BB4A009998328918BA4A914203D25B
:10FE1000B94A0299914200DD0120297F012921D0B0
:10FE2000012832D0B049A288E839C888801A00B2C7
:10FE3000002801DAB14A801800B2C82811DCEE832C
:10FE400008780928208827D0401C208000B20A2882
:10FE500007DD01202877A071E079012801D1A96A86
:10FE60008847FEBD012F01D0EE83FEBD9E48E838D5
:10FE700000780928E88B06D0401CE88300B20128EE
:10FE8000F3DD2E77FEBD401DF7E70020205E002841
:10FE9000F8DD401E2080FEBD401DD6E7924B083B9A
:10FEA000642809DA642A07DA90487D380818C728D8
:10FEB00002D25888401C58809888401C988070470F
:10FEC00010B5894C0823E83CE356012B15D0022BD2
:10FED00015D0032B16D0042B16D0002800DC40428E
:10FEE00000B2002900DC494209B2002A00DC52427B
:10FEF00012B288420BDA0B460AE0400000E04800EC
:10FF000004B214E05000FBE740188018F8E70346FD
:10FF1000934201DA134604E0884201DA0B4600E01E
:10FF200003461B185B189B181CB2FFF7B7FF20464F
:10FF300010BDF8B50F46054616463843304321D06C
:10FF4000694C1C20883C205E32281ADC2846FFF7CA
:10FF5000B7FF1C21615E22464900603A8918603172
:10FF6000C883324639462846FFF718FF32463946DD
:10FF70002846FFF7D4FEA08B401C00B2A083322895
:10FF800001DB0120F8BD0020F8BD574810B538212D
:10FF9000123000F0DEFE54490E20E839C881524884
:10FFA0000F214030817240384168012903D0FF2180
:10FFB000D731018110BDFF21A531FAE7FFB50C460D
:10FFC0004F1005464849FF205F30CE8C81B08442F7
:10FFD0000EDC039813280BDB0C2E01D3AF4226DC7A
:10FFE0000321204600F058FEA84201DB082E1ED255
:10FFF0002046FF386038F92808D80398112805DB17
:020000040002F8
:10000000AF4214DA0C2E01D3A54210DB37483C492D
:10001000C7302018884208D203980C2805DBAF426D
:1000200005DA0C2E01D3A54201DB142E02D90120E2
:1000300005B0F0BD0020FBE72B48C08C08280FD38B
:10004000132A03DCFF205F30814207DB112A03DC27
:100050004B20C000814201DB0C2A01DA01207047ED
:1000600000207047F0B5204D1F49883D1826AE5F2F
:10007000488D8FB0301A00B203904E85002867DBA0
:10008000002042005218D38D9385401C138B40B240
:10009000D3820728F5DB1620285E0B9048878E84D4
:1000A0002820085E082801DA401C088500200E4937
:1000B00004900190282402460C5F07200823191B96
:1000C0008C4631E0430059182C232A27CB5ECF5FA2
:1000D0009E46FB1A002B01DC7346DB1B049F5B1062
:1000E000DF19BFB273460DE0C0360020E0FCFFFF11
:1000F00056020000E903000070FEFFFF30750000AB
:10010000C74B0000DB1004979A1816231427CB5E08
:10011000CF5F92B2D91B002900DCF91A019BC918E4
:1001200009B2401E40B20191FE498445CADB41003C
:10013000FC4808182C21415EC810801880B2214666
:1001400000F0AAFD8004070C022C02DAF54846856F
:100150004CE0611E049800F09FFD4600611E01986E
:1001600000F09AFD00B284460B98009039B230B28C
:1001700062460C460646039BFFF75EFF002802DD41
:10018000FFF703FF32E0E748817C002908D0C18FE8
:100190003A0A8918C187298B418501200FB0F0BD2B
:1001A0000746C08C401C80B2F884082805D2132171
:1001B0007956002918DD032816D9624621463046B3
:1001C000039BFFF7FBFE00280EDD0120B874D54825
:1001D000142140308172FF205F303881F88CF97C27
:1001E0004018401C40B2D9E7288B78850020D5E71D
:1001F00070B5CC4C01202056002804DDFFF732FFFB
:10020000218A40182082C74DE08C4035002826D036
:100210002E46C83E308B618D401A00B2002802DAAB
:10022000C149401800B26E2804DDFFF7AEFEE08C35
:10023000002814D00A2170886956884202DCA889F7
:100240006E280CD91620305EFF21D731884204DD9C
:10025000FFF708FF218A40182082FFF796FEB14879
:100260003221E838C08800F001FD00291DD1A07CB2
:1002700000280AD0E08C002814D004210620695EF2
:10028000285E0A1A052A07DA08E004210620695EBA
:10029000285E0A1A042A01DB022801DB082901DB97
:1002A000FFF773FE0020A880E880002070BD9D4805
:1002B0004030007D042801D00020704701207047A5
:1002C000F8B5024697480021E83806467C360546D0
:1002D00034460835EC34012A1ED00A220270074643
:1002E0004180FFF752FE5021284600F032FD6A217E
:1002F000304600F02EFD0E20F8818A490820C8748F
:1003000005202056002806DDA268002A03D0002020
:10031000385600219047F8BD0922027041800746F7
:100320005021284600F015FD6A21304600F011FDED
:10033000E6E77C4910B588394A8800206039102AE0
:1003400001D900224A80774A0023D356002B01DDD1
:10035000CB888B800B78092B0AD0CA888988511AE0
:1003600009B2FA2903DD0120FFF7AAFF012010BD21
:100370000123D356002BFADD4A88521C92B24A80E0
:10038000042AF4D90020EFE7664980310A7B012A6C
:1003900001D1096908477047FEB501460026FFF7FD
:1003A00086FF604C00276034012802D02772304657
:1003B000FEBD208B401C20835A48498802460546D2
:1003C0006E326930803500920190002909D0E08AB0
:1003D000401CE0820820205607284ED0062833D043
:1003E0004BE0A08A401C01B2A182082020560628BA
:1003F000DDD0002815D00728D9D1022909DA4948CB
:1004000094300290FFF7C0FF05220299009800F097
:1004100087FC1420205E1428C9DDA07F012804D0A9
:1004200009E01429C3DD062029E008202B682056A6
:10043000009A0199984706202072A08BE18A401803
:10044000A0830126E782B2E70198FFF79DFF142001
:10045000205E14280EDDA07F012805D108202B681E
:100460002056019A00999847608BA18A012640186E
:10047000608302E0A18B0818A083A7820720207266
:1004800095E770B5274800244030448384830546AF
:10049000C48320352C801621283000F05AFC2C72A1
:1004A00070BD204817218030415609390B2901D3EE
:1004B000012070470020704770B50246FFF7F7FE35
:1004C000184C4034002834D1FFF7EBFF012830D11D
:1004D00050880A282DD210881E282AD20120607444
:1004E000FFF7CFFF042021462075403105228A56B0
:1004F0000025002A05DD8A68002A02D000219047E5
:10050000E582084862300646FFF73EFF05480522AF
:100510006030858231460E3000F002FC0522314603
:10052000004803E0C036002030750000693000F05C
:10053000F7FB1420205670BD70B5F948417C0029A6
:1005400010D01E25818B455F0824481900B20C2865
:1005500006DB0A2100F0A0FB00B2854200DB052487
:10056000204670BD052070BDF8B50546FFF7E4FFD5
:10057000EB4E05213446307540346156002904DDC8
:10058000A268002A01D029469047E5485430074622
:10059000FFF7FAFEE24D14202035285E0F28A87FD1
:1005A00007DD01280DD129460E313A460620236881
:1005B00006E0012805D1DA49236829313A460720A7
:1005C000984700202872A87F012806D11420D4491A
:1005D000236830563A4622319847F8BD10B5FFF7E8
:1005E00066FE012820D1CE488030C188282918D83D
:1005F00081883C2915D84189642912D80189FA29B2
:100600000FD8C189C8290CD88089FF21913188422F
:1006100007D8FFF746FF002806D1FFF78DFF052812
:1006200002D00020FFF7A0FF10BD70B50246FFF713
:100630003EFE0025BA4C012804D06575E5821520E0
:10064000205670BDB6495088203102280AD2A08BAE
:10065000401CA083607D072802D10888401C0880C8
:10066000062009E0E08B401CE083607D062802D173
:100670000888401C088007206075A9480521403083
:1006800041560029DADD8368002BD7D002211520DE
:10069000515E20569847D1E770B50446A04D122010
:1006A0002856002802D001280AD00FE0012C0DD1D5
:1006B000FFF7FDFD012809D10020FFF755FF05E0F8
:1006C000002C03D19649002040398881AC7470BD5C
:1006D00010B5934C0420483C205E64280CDD0221B8
:1006E000615E401A052801DA012000E00020FFF7D2
:1006F000D3FF00206080A08010BD70B588484030D6
:100700000079002831D0864D0521403DA88900F0B0
:10071000ADFA834C00290BD1207C012802D0607CEB
:10072000012801D1FFF7D4FF7D488830FFF77DFF16
:10073000A8890A2815D9207C012802D0607C0128CC
:100740000BD1FFF74BFF207C012806D1A07C0028AD
:1007500003D173488C30FFF7AFFE71488430FFF748
:100760001BFE6F4858300021C16270BD10B56D4846
:10077000007809280AD06A4880304188142905D2B7
:1007800000881E2802D20120FFF79AFD64494039F3
:100790000F20085610BD70B561490023403958003C
:1007A00040180246C032548AE0301482C2888280E7
:1007B0005B1C428B1BB20283092BF0DB58480024E0
:1007C000803002460388203253804388D382483ADF
:1007D000092314635A005218D0260589B65AE0320C
:1007E000AD190581458992885B1EAA181BB242810A
:1007F000052BEFDA4A4A5832092354635A0052183B
:10080000D0248589A45AE0322C198481C489928825
:100810005B1EA2181BB2C281002BEFDA70BD10B5AF
:1008200040480278E8304189092A22D0491C418198
:100830008AB23D498A421AD98289521C92B2828177
:100840008A4201D96421818100244481FFF7A3FFFA
:10085000FFF78CFF32485430FFF796FD30480121F6
:1008600040300171014618318A6A8C62CA620020E8
:1008700010BD491DDBE74188C180704710B50028D5
:1008800001DD034600E043421CB2264B94420CDAE1
:100890001C78092C4C8906D0641C4C81002806DA8F
:1008A0000020C04310BD641DF7E70024F5E7904227
:1008B00008DD02228A5E824204DA4880D8880881F4
:1008C000012010BD002010BD70B50C460021615EF6
:1008D0000025002902D0022914D108E03C2221463B
:1008E000FFF7CCFF00280DDD022020800AE03C222B
:1008F0002146FFF7C3FF002804DA6088E0806581A5
:10090000012070BDA088401C00B2A080802805DBBB
:100910000C21204600F01DFAA5802580002070BD26
:1009200000370020D8350020B80B0000F8B5CC4CBB
:1009300021782046C088092955D0401CE080C9494B
:1009400080B20025884200D9E580C5490A20205E92
:10095000583100270091FFF7B7FFC14E60360028DD
:100960000CDD304601270C221030009900F0D8F938
:10097000032030820C21009800F0EBF9B8490C20DC
:10098000205E64310091FFF79FFFB74C00280ADD1D
:100990000A20305E642802DDA088401CA0800C2163
:1009A000009800F0D6F9A089401CA081AE484038DC
:1009B00045700570002F14DD0146C0310A880123FF
:1009C000521C0A8003701622B25E0826865FB2426D
:1009D00007DDE288521CE2804A88521C4A80A581C9
:1009E00043703846F8BD401DA8E770B5531E1D463C
:1009F0001E2B20D2002305E05C00661876885B1C65
:100A00000E535BB2AB42F7DB831050004018203826
:100A1000C3830020521053B2024608E0D418640089
:100A200055000C5F4D5F641B2018521C52B29A4255
:100A3000F4DB002B01DC002071E7194600F02CF9F3
:100A4000800000B26BE730B5002253005C18521CE6
:100A5000648852B2CC52032AF7DB0022C8800223FA
:100A60001046C418450064000C5F4D5F401C641BB9
:100A7000A21840B29842F4DB501000B230BD70B5FD
:100A8000774C0646207809280ED00E22A25E30460A
:100A9000FFF7ABFF0546214606224C313046FFF7F3
:100AA000A4FFA08128463AE73046FFF7CCFF054671
:100AB000F8E7FEB56A4C6C4E0021403E204631827C
:100AC0001030274601906037FF3059300D460090B6
:100AD0001FE0680001197E20085E0199FFF7CFFF33
:100AE0006081FFF723FFFFF79AFEFFF706FEFFF78F
:100AF00020FC002811DCFFF7DAFB012804D0207865
:100B0000092801D0FFF774FB002000996D1C0871C3
:100B10002DB21C20385EA842DBDC0020B8831020F8
:100B2000B18A305E0918B182FEBD4F4940318860FC
:100B300001204871002070474B4940310861012075
:100B40000873704748494031086047480121203008
:100B500081777047444940390F200856704700207C
:100B6000704741494039012804D0FF22D7320A8119
:100B700048607047FF22A532F9E770473A4A2823B8
:100B8000403AD35E042B07DB820012B2814201DBC4
:100B9000914201DD0120704700207047012070471D
:100BA00070B5314C05000DD1207C01280AD1FFF72A
:100BB0007EFB012806D1FFF7BFFC052802D00020EC
:100BC000FFF7D2FC2574AAE670B5274D0024403DFE
:100BD000012807D0FFF76BFB012802D1FFF7C4FC07
:100BE000AC819CE6FFF763FB0028FAD11E4E7474BB
:100BF000AC8141004919D0225452E031401C8C8014
:100C000000B20C830A28F4DBFFF73BFC16490420F2
:100C10003075403105228A56002AE2DD8A68002AB2
:100C2000DFD000219047F48279E60F494031886295
:100C30000D4801216030C17170470B4901226031BC
:100C40000A7300220A824A828A82CA82C881704755
:100C500005494031C863044801216030017670477E
:100C6000D8350020307500000037002030B50B4625
:100C7000014600202022012409E00D46D5409D4276
:100C800005D31D469540491B2546954040191546FC
:100C9000521E002DF1DC30BD70B500242546002821
:100CA00001DA01244042002901DA01254942FFF717
:100CB000DDFFAC4200D04042002C00D0494270BD64
:100CC000F0B51FB40646002082B0054640240191CD
:100CD00000901BE0019922460F46304600F068F86C
:100CE000049A059B801A994110D310461946224652
:100CF00000F04EF8361A8F4101972246012000215C
:100D0000009F00F045F838184D4100902046641EC1
:100D10000028DFDC019B00982946324607B0F0BD71
:100D200003460B439B0703D009E008C9121F08C004
:100D3000042AFAD203E00B78491C0370401C521EAF
:100D4000F9D27047D2B201E00270401C491EFBD2BA
:100D500070470022F6E710B513460A4604461946C6
:100D6000FFF7F0FF204610BD421C0178401C00290F
:100D7000FBD1801A704730B504460020034600E0DE
:100D80005B1C934203D2E05CCD5C401BF8D030BDCD
:100D900010B5202A04DB0146203A9140002010BD06
:100DA000914020239C1A0346E3401943904010BD14
:100DB00010B5202A04DB0846203AD040002110BD9F
:100DC0000B46D340D0402024A21A91400843194634
:100DD00010BD0000064C0125064E05E02046E368E4
:100DE00007C82B4398471034B442F7D3F5F76CF992
:100DF000442402006424020070B58C180578401C5D
:100E00006B075B0F01D10378401C2A1106D10278D1
:100E1000401C03E00678401C0E70491C5B1EF9D193
:100E20002B0705D40023521E0DD40B70491CFAE782
:100E30000378401CCB1A921C03E01D785B1C0D70DC
:100E4000491C521EF9D5A142D8D3002070BD000024
:100E50000FB410B504A9074B02AA039800F028F8B4
:100E6000044602A9002000F061FA204610BC08BC2C
:100E700004B018472D13020030B47446641E257860
:100E8000641CAB4200D21D46635D5B00E31830BCBE
:100E9000184702E008C8121F08C1002AFAD170479B
:100EA0007047002001E001C1121F002AFBD17047EA
:100EB000FFB591B00F4605460026F9E0252876D10A
:100EC00000246D1CFB4A0094012102942B780846F3
:100ED000203B98400346134202D004436D1CF5E7C3
:100EE00028782A280ED0022128780246303A092A8A
:100EF00015D8009A0A235A43303A80180C436D1CC7
:100F00000090F1E701CF0090002805DA01204003AE
:100F10000443009840420090022004436D1C28784E
:100F20002E2815D1042004436D1C28782A280AD1C4
:100F300001CF6D1C02900BE002990A225143303917
:100F400040186D1C02902878014630390929F3D9E0
:100F500028786C2810D006DC4C281AD068280ED0CF
:100F60006A2817D104E0742813D07A2812D110E02F
:100F70000120400504430CE00121090501E00321A3
:100F800009050C436978814203D101206D1C0005DD
:100F900024186D1C287803906E281FD00DDC632860
:100FA00033D005DC00287DD0582812D1BEE010E0F7
:100FB000642801D069280CD181E073282FD004DC8B
:100FC0006F2870D0702804D1B2E075286CD07828D2
:100FD0006BD0149A13999047761C68E06002400F1A
:100FE000022807D003280AD0042838680AD03F1DF9
:100FF00006605CE001CFF1170660416057E001CF69
:10100000068054E03F1D067051E038786946087448
:101010000020487404A83F1D0390012003E001CF85
:1010200003900020C04361070FD5002101E0019922
:10103000491C029A0191914213DA8142F7DB019A2D
:101040000399895C0029F2D10BE0002101E00199AC
:10105000491C01918142FADB019A0399895C0029BC
:10106000F5D101990098139A401A00902146149BDB
:1010700000F046F901998019461807E00398039992
:101080000078491C0391149A139990470198401EC7
:101090000190401CF2D12146149B139A009800F055
:1010A0001FF903E008E04CE03EE03FE086196D1CCC
:1010B0002878002800D001E7304615B0F0BD0A209E
:1010C0000021049005916002410F022905D001CF53
:1010D000C2179446032907D009E0FF1DFF08FF004F
:1010E00079683868083706E000B2C21794460429C8
:1010F00002D140B2C1178C4600226146944506DAFF
:101100000A460021404291418C462D2102E02105F2
:1011100004D52B216A461176012103E0E10701D0B5
:101120002021F7E7019150E00A200BE0102009E0B0
:10113000102004900021042004430820059102900F
:1011400003E008200021059104906002410F02296C
:1011500005D001CF00229446032908D008E0FF1DE6
:10116000FF08FF007968386808378C4603E080B2D2
:10117000042900D1C0B200210191210725D503998E
:1011800070292AD0049A1021059B4A401A4309D19C
:101190006146014306D030216A46117603995176A3
:1011A00002210191049A0821059B4A401A430CD15F
:1011B0006146014301D1610707D530216A461176A6
:1011C000012101910299491E02910399582909D0E0
:1011D00039A103910FA90F9112E040216A461176BF
:1011E0000121DEE739A1F4E76146059B049AFFF788
:1011F00067FD039B8C469B5C0F9A521E0F921370E7
:1012000061460143F0D10F9807A9081A20300390D6
:10121000600704D5012000048443029801E0012006
:1012200002900399884201DD401A00E00020411835
:101230000290019809180098401A0090E00306D423
:101240002146149B139A009800F05AF88619002042
:1012500007E006A9085C149A139990470498761C35
:10126000401C019904908842F3DBE0030CD5214631
:10127000149B139A009800F043F8861904E0149A1E
:10128000302013999047761C0299481E029000293D
:10129000F5DC08E00F980F990078491C0F91149A1B
:1012A00013999047761C0399481E03900029F1DC9E
:1012B000F1E6000009280100303132333435363789
:1012C0003839616263646566000000003031323392
:1012D0003435363738394142434445460000000032
:1012E000F8B5044600251E461746880404D405E0D8
:1012F00039462020B0476D1C641EF9D52846F8BD3C
:10130000FFB50446002581B01E46C80301D530272D
:1013100000E02027880404D505E038460399B0474B
:101320006D1C641EF9D5284605B0F0BD0A68531C33
:101330000B6010707047000070B50D46FEF740FB63
:10134000040004D1FF2103A28A31F4F783FF256250
:1013500070BD00002E2E5C2E2E5C2E2E5C2E2E5C80
:101360002E2E5C536F757263655C7370695F6D617F
:10137000737465725C7370695F6D61737465722EEE
:1013800063000000216401006D6201004B640100F4
:101390006D620100CB6401006D620100E8E8E8E8DD
:1013A0001717171700000000101819120408080872
:1013B000101010101010080808041219181000005E
:1013C0000000000000000F7080000000000000001E
:1013D000000303081020408000000080700F000010
:1013E0000000000003C03C040201000000000000F7
:1013F0007C7C00000000000003060438C0030000ED
:10140000000000C02020202080804040402020207C
:10141000202020404040800020202020C0000000EC
:101420000000000000000000001010111111111F39
:1014300011111100001F1F0000000000000000003B
:10144000000000000000003F7FE0EFCFDFDFDFDCC7
:10145000DCDC1C1CFCF800000000000000000000A8
:10146000000000000000E0E000FCFDFDFCF80000D2
:10147000000000000000000000000000000000006C
:101480000000000000000060F0F8F8F060000000CC
:10149000000000000000000000000000000000004C
:1014A000000000000001010000000000000F3F3FAD
:1014B0007F7F3F3F1F07000000000000000000008A
:1014C0001E7EFEFEFEFEFEFE3C00000000838787BF
:1014D0008787878783000000000000000000000F5E
:1014E0001F1F1F1F1F1F0F0301007CFEFFFFFFFFB9
:1014F000FFFFFEF800000000000000000000E0F820
:10150000FCFEFEFEFEFEF8F0000000808080808081
:1015100000000000000000000000000001232F3E3A
:101520003E2F232120202030383C3F1F0F00000099
:101530000000000000000000000078FEFF870707A1
:1015400087FFFE78000E1F3870E0C08000000000AA
:10155000000000000000000000000000000000008B
:1015600000000000000080404043475F7C7C5F47F4
:101570000300000000000000000000000000000068
:1015800000000000000000F0FCFE0E0E0E0EFEFC3F
:10159000F000000000000000000000030707081032
:1015A0002020202020202010080F07030100000029
:1015B00000000000000000003FFFFEFCFF7FFF1F57
:1015C0000F0703003F1FFFFFFFFFFFFCC0000000ED
:1015D0000000000000000000C00000E0F8FCFEFE7B
:1015E000FFFFFFFFFFCFE3F0F880000000000000E6
:1015F00000000000000000000000000000000000EB
:1016000080C0FCF0C00000000000000000000000EE
:1016100000000102040808080403010000000000A3
:1016200000000000000000000000000000000000BA
:1016300000E0180601000000069B71000000000099
:10164000000000000000000000000000000000009A
:1016500000000000804020100884C26130180C0493
:10166000040C0808080C040203010000000000003C
:10167000000000000000000000000080402010106A
:101680000808080808081830E00000000000000002
:10169000000000000000000000000000000000004A
:1016A000000000000000000000000000000000003A
:1016B0003F302824222120212222222222212021DF
:1016C000222428303F00000000000000000000FE3F
:1016D000060A12224282020202020202028242220E
:1016E000120A06FE000000000000000000000000DA
:1016F00000000000000000000000000000000000EA
:1017000000000000000000000000000000000103D5
:1017100007070F0F1F1F1F1F1F1F1F1F0F0F070779
:10172000030100000000000000000F3FFEFCF8F085
:10173000E0E0E0C0C1C1C1C1C1C0E0E0F0F8FCFF21
:10174000FFFF3F0F0000000000F0800000000000DD
:101750000000101090503000000000000003FFFF58
:10176000FFFCF00000000000000000000888C8A88E
:101770009880000000000000081870E0E0C08000C1
:101780000000000000000000000000000000000059
:101790000000000000000000000001020100000045
:1017A0000000000000000000030408101727272590
:1017B0002527271710083C4B881020408000000088
:1017C000000000000000FC03000000FE0202020214
:1017D0000203FE00000003FC000000000000000007
:1017E00000000000000000804020201010101010A9
:1017F00010202040800000000000000000000000D9
:1018000000000000000000000000000000000000D8
:1018100000000000000001020100020100010200BE
:101820000000000003040810172727252527271785
:1018300010083C4B88102040802040804020000051
:101840000000FC03000000FE020202020203FE0090
:10185000000003FC00000000000000000000000089
:101860000000008040202010101010101020204098
:1018700080000000000000000000000000000000E8
:1018800000000102020606060C0C0C0C0C0C0606ED
:1018900006020201000000000000000000031F7C9F
:1018A000E0800000000000000001010000000000D6
:1018B000000080E07C1F030000000000F0FE0F012C
:1018C0000000000000000000FFFF0000000000001A
:1018D0000000010FFEF00000000000000080C0606A
:1018E00030300000000000F8F80000000000303048
:1018F00060C0800000000000000000000102041829
:101900002020202020202020201806010000000098
:101910000000000000000000000000F008080700C0
:1019200000030101010202020404F80000000000AB
:101930000104020100000000001F000F00F905056E
:10194000FD017F6060FBFBE0FFE2E2FFFFFF7F3F06
:10195000807C00FE00000000E010C82490C0E0E0A1
:10196000E0E0E0E0E0E0E0E0E0E0E0E0E0C08000D7
:1019700000000000000000000102041820202020C8
:101980002020202020180601000022140814220024
:1019900000000000000000F008080700000301013B
:1019A000010202020404F800000000000104020128
:1019B00000000000001F000F00F90505FD017F6019
:1019C00060FBFBE0FFE2E2FFFFFF7F3F807C00FE69
:1019D00000000000E010C82490C0E0E0E0E0E0E09B
:1019E000E0E0E0E0E0E0E0E0E0C0800000000000D7
:1019F00000000000010101010101010101010101DB
:101A000001010101010101010101010000000000CB
:101A1000007FFFFF80808080808081828484848436
:101A2000848281808080808080FFFF7F00000000B2
:101A3000FEFFFF010101010100E0100F0F0F0F0F6A
:101A400010E0000119191901FFFFFE00000000005D
:101A50000080C0C0C0C0E0F07070707070707070B6
:101A600070F0E0C0C0C0C080000000000000030FA4
:101A700009191F39393F3F3F1E1E0E0F0703010092
:101A8000000000000000000000000000F8FEFF3F22
:101A90003FF83020C080000000000080C0E0F078F7
:101AA0003C1E0F0703010000000000000080C0E0A2
:101AB000F0783C1E0F070301000000000000000149
:101AC00002068FDEFEFF3F0F000000000000000056
:101AD0000000000080C0E0F078381C3C7EFEFE4E26
:101AE0004EFC4C48F8E00000000000000000000040
:101AF000000000000008080F0F08080000000000A8
:101B000000000000000000000000000000000000D5
:101B100000001F204F5F5F5F5F4F201F000000002D
:101B200000000000000000000000000000001F0096
:101B3000000E01FCFEFEFEFEFC00000000000000A6
:101B400000000000000000000000000000804020B5
:101B500010109090900000000000000000000000B5
:101B6000000000000000000000000102040408085A
:101B70000818181F1F18180808080404020100009C
:101B80000000000000000738C000804020001F2037
:101B90004F5F5F5F5F4F201F0000000000C03807ED
:101BA0000000000000E01C0300000000000000FC3A
:101BB000FEFEFEFEFC00020100000000031CE0002F
:101BC00000000000000000804020201010100808D5
:101BD00008080808101010A0204080000000000035
:101BE0000000000000000000000000000008080FD6
:101BF0000F080800000805020508000000000000AA
:101C0000000000000000000000001F204F5F5F5F29
:101C10005F4F201F800000008000000000000000D7
:101C20000000000000001F00000E01FCFEFEFEFE92
:101C3000FC000000000000000000000000000000A8
:101C400000000000008040201010909090000000E4
:101C5000000000000000000000000000E0180C1E62
:101C60003A71E1C1C1E1713A1E0C18E000000000B8
:101C70000000000000000000000000071830785C41
:101C80008E878383878E5C78301807000000000001
:101C90000000000000000000000000000000102014
:101CA0004080FC8CD8702000000000000000000084
:101CB0000000000000000000000000000008040216
:101CC000013F311B0E040000000000000000000076
:101CD0000000000000000000000000C08004149418
:101CE00024489020C0000000000000000000000018
:101CF000000000000000000000003B24292A0C081E
:101D000000010003000000000000000000000000CF
:101D10000000000000000000001F10101010101044
:101D200010101010101010101010101010101010B3
:101D30001F03000000000000F80808080808080851
:101D4000080808080808080808080808080808F823
:101D5000C00000000000001F101010101414141414
:101D600014141717161410101010101010101F0351
:101D7000000000000000F8080808080808082868A3
:101D8000E8E8E868282828280808080808F8C000B3
:101D900000000000000000FE78C078FEFE00FCFE9F
:101DA0000202FEFC00FE38C0FEFE00000000000043
:101DB00000000000000007000100070700030704FF
:101DC00004070300070001070700000000000000EF
:101DD0000000000606F6F6060600FEFE0000FEFE07
:101DE00000FC66666606007C666666E6000000002B
:101DF00000000000070700000003070404070300B9
:101E0000030606060600060606060300000000009C
:101E1000000000FEE018E0FEFE00FC666666660656
:101E200000FE020202FCF8000000000000000000BA
:101E3000000007010001070700030606060606006A
:101E4000070404040301000000000000000000007B
:101E5000000606F6F6060600FE606060FEFE00FE66
:101E6000000000FEFE00FE46C6C67E000000000028
:101E70000000070700000007000000070700030438
:101E8000040407030007000001030000000000FE37
:101E9000666666660600FE46C6C67E38000000FE20
:101EA000FE0000000000000000000000000007002D
:101EB0000000000000070000010306000000070703
:101EC000000000000000000000000000007C6666CA
:101ED0006666E60000F04E4EF000000606F6F606D6
:101EE00006000000000000000000000006060606D4
:101EF00006030007000000000700000007070000BD
:101F000000000000000000000000007C66666666BD
:101F1000E600FE000000FEFE00FE38C0FEFE0000EF
:101F20000000000000000000000006060606060390
:101F30000003040404070300070001070700000072
:101F4000000000000000000103060C0C0C0C0C0C3F
:101F50000C0C0C060301000000FFFFFF0000000056
:101F60000000000000000000FFFF0000FEFFFF0077
:101F70000000000000000000000001FFFE00000063
:101F80000080C0606060606060606060C080000071
:101F90000000000000000000000000000F0F0F0014
:101FA000000000000000000000000000000000FF32
:101FB000FFFF000000000000000000000C0E0703FF
:101FC0000100FFFFFF000000000000000000000013
:101FD000000080C0E0E0E0E00000000000000F0F23
:101FE0000F0C0C0C0C0C0C0C0C0C0C0C0C0C0C003A
:101FF00000E0F0F818181818181818181818181CF5
:102000000F0700001E1F1F0000000000000000005E
:10201000000001FFFE0000000080C06060606060A2
:1020200060606060C08000000000000103060C0CCE
:102030000C0C0C0C0C0C0C060301000000E0E0E0A2
:10204000000001010101010101010101FEFC00008C
:102050000607070000808080808080808080817FEC
:102060003E0000000080C060606060606060606092
:10207000C080000000000000000000000000000020
:1020800000000F0F0F000000007E7F636160606042
:102090006060606060FFFFFF60600000000080C063
:1020A000E070381C0E070301FFFFFF000000000076
:1020B00000000000000000000080C0E0E0E0000040
:1020C0000000000103060C0C0C0C0C0C0C0C0C0694
:1020D0000301000000C0C0C00000000000000000BC
:1020E00000000000FFFF00007F7F7F606060606095
:1020F00060606060606060C0800000E0E0E06060A0
:1021000060606060606060606060600000000001AE
:1021100003060C0C0C0C0C0C0C0C0C060301000040
:1021200000FFFFFF000000000000000000000000B2
:10213000FFFF0000FEFFFFC0C0C0C0C0C0C0C0C0E5
:10214000C0C0C183020000000080C06060606060A9
:1021500060606060C08000000000000000000008B7
:102160000E07010000000000000000000000000059
:102170000000000080E0781E070100000000000061
:10218000000000000000000000000080E0781E0752
:10219000010000606060606060606060606060605E
:1021A0006060E0E00000000103060C0C0C0C0C0C5D
:1021B0000C0C0C060301000000F8FCFC03030303F5
:1021C0000303030303030303FCF800007EFFFF0087
:1021D0000000000000000000000001FF7E00000081
:1021E0000080C0606060606060606060C08000000F
:1021F0000000000103060C0C0C0C0C0C0C0C0C0663
:10220000030100000081830706060606060606068F
:1022100006060606FFFF0000FEFFFF0000000000AC
:1022200000000000000001FFFE0000000080C06010
:102230006060606060606060C0800000000000005E
:102240000000000000000000000000000060F0F04E
:102250006000000000000000000C1E1E0C000000CA
:102260000000000000000000000000000000000E60
:102270000F0100000000000000000000C0F83F0750
:102280000000000000000000000000E0FC1F030050
:1022900000000000000000000080F070000000005E
:1022A0000000000000000000000000000060F0F0EE
:1022B00060000000000000000000000000000000BE
:1022C00000000000000000000000000032003200AA
:1022D00002002003030064006400020020030600E3
:1022E00096009600020058020600C800C8000200CE
:1022F00058020600000000801200000014000000D8
:1023000011000000130000000100000000010100A6
:10231000000001020406090C1014181D23282E3594
:102320003B424A51586068707880889098A0A8AF66
:10233000B6BEC5CBD2D8DDE3E8ECF0F4F7FAFCFE8C
:10234000FFFFFFFFFFFEFCFAF7F4F0ECE8E3DDD857
:10235000D2CBC5BEB6AFA8A09890888078706860D0
:1023600058514A423B352E28231D1814100C0906DB
:10237000040201000308090A000102030405020324
:102380000000D0002D121E4B0FA4994ECEB531F493
:102390000579D9D9AAFDBD9B2198A849E145F3D873
:1023A000D169BD1DA299E625588CD94201630D1251
:1023B000BF9FFB7B7CCE6AB344BEB54BD624E9C637
:1023C000EA22000031F501006FE8010035F5010057
:1023D00039F5010041F5010001E9010045F5010071
:1023E00049F5010051F501002DE9010055F5010005
:1023F00059F501002E2E5C2E2E5C2E2E5C2E2E5CAE
:102400002E2E5C536F757263655C626C655C6465EF
:10241000766963655F6D616E616765725C64657640
:102420006963655F6D616E616765725F7065726932
:1024300070686572616C2E6300000000020000008D
:10244000000000006424020000200020840300003B
:10245000F80D0200D4250200842300204C1C00004B
:10246000A20E020011A324F4A201CBFFFF10D91F7A
:102470000112491D051122FF420E23070319031102
:102480003C4F6B010841149D69019A040C0716101A
:1024900027AF32011214ED8501142188011ABB0403
:1024A00014EF8A0114558B0114578C011AA70414D8
:1024B000018E011A810414878F011AD704145190D8
:1024C000011AD90414919101141392011A89041468
:1024D0002993011ADB04142F9401147D95011AC16C
:1024E00004143B97011A7F0414F59801143D9901D7
:1024F000145B9A011A8D0414499B011A8F04140568
:102500009C011A79040B1B639DF60119147D1F02AF
:102510001AC904141520021A61041AAD041AF90428
:10252000144521021A91041ADD04142922021A60AA
:10253000041A90041AC0041A6A301AB6041A02283F
:102540001A4E041A9A041AE6041A322C1A7E041A35
:10255000CA041A16281A54041A84041AB4041A57FE
:10256000301AA3041AEF041A3B2C1A87041AD30456
:102570001A1F2C1A6B041AB7041A03281A48041AD3
:1025800078041AA8041A442C1A90041ADC041A2895
:102590002C1A74041AC0041A0C2C1A58041AA40415
:1025A0001AF0041A3C2C1A6C041A9C041102130829
:1025B00072010E11282E323C3E1F161049352B3564
:1025C000140201017A04141C8020014E09184C01E8
:0425D000F300000014
:00000001FF
